:020000040800F2
:104000000050002059D5000869B000086BB00008C6
:104010006DB000086FB0000871B00008000000002B
:1040200000000000000000000000000075B0000863
:1040300073B000080000000077B00008CD820008CF
:1040400079B000087BB000087DB000087FB00008A0
:1040500081B0000883B0000885B0000887B0000870
:1040600089B000088BB000088DB000080000000087
:104070000000000000000000000000000000000040
:1040800000000000000000009DB000089FB0000884
:10409000ADB00008BDB00008CDB00008DDB000082C
:1040A000DFB00008E1B00008E3B00008E5B00008A8
:1040B000E7B00008E9B00008EBB00008EDB0000878
:1040C000EFB00008F1B00008F3B00008F5B0000848
:1040D000F7B000083D810008FBB00008FDB0000803
:1040E000FFB0000801B1000803B1000800000000A3
:1040F00000000000000000000000000000000000C0
:0C41000000000000000000005FF800005C
:1041100030BF704720BF704740BF7047BFF36F8FFD
:104120007047BFF34F8F7047BFF35F8F704701DF5A
:104130007047EFF31480704780F31488BFF36F8FDC
:104140007047EFF30980704780F309887047EFF3F9
:104150000880704780F30888704772B6704762B66F
:10416000704771B6704761B6704780F31188704729
:10417000EFF31280704740BA704700BA70470000F2
:104180002DE9F3414B4E4C48012107F0EDFD042091
:10419000012108F0D1F80324102542F21203304621
:1041A00001A94FF00408ADF804308DF807508DF8E0
:1041B000064007F04AFD02233561404F73613046E7
:1041C0004CF204430DEB0801ADF804308DF80640C5
:1041D0008DF8078007F039FD0820012108F0ACF8C0
:1041E00041F61C7338460DEB0801ADF804308DF82C
:1041F00007508DF8064007F028FD4FF4F8533B6157
:104200000C237B613846E0230DEB0801ADF8043048
:104210008DF806408DF8078007F017FD284601212C
:1042200008F08AF88DF80750254D4FF46043284672
:104230000DEB0801ADF804308DF8064007F005FDE0
:104240004FF420432B614FF480436B614FF4805354
:10425000ADF80430284648230DEB08018DF80730EF
:104260008DF8064007F0F1FC0121164807F07CFDAF
:1042700000230A211A464FF400507061B46830617F
:10428000B068640458BF0132400448BF01330139AB
:10429000F1D10A2A0C4A03D10A2B01D1012300E0F3
:1042A000002305480121137007F05EFD02B0BDE850
:1042B000F08100BF0008014000023000000C014006
:1042C0000010014000043000740E0020124B82B038
:1042D0001B78F3B1114B4FF400725A614FF48072A6
:1042E0001A610022019201990D4A914202D8019A65
:1042F0000132F7E74FF400721A614FF480725A618D
:1043000000230193019A064B9A42E3D8019B0133A3
:10431000F7E702B0704700BF740E0020000C0140A8
:104320003F0D030010B1012802D07047082200E0C1
:104330000422014B5A617047000C014010B1012862
:1043400002D07047082200E00422014B1A61704736
:10435000000C014038B50546002445FA04F3DB079C
:10436000E0B202D5FFF7EAFF01E0FFF7DBFF01341F
:10437000082CF2D138BD08B504281ED8DFE800F0BB
:1043800003050A0F140000200FE00D4B9868C0F3DE
:10439000801008BD0A4B9868C0F3C01008BD084BD8
:1043A0009868C0F3401008BD042004F07FF8B0F511
:1043B000006F94BF0020012008BD002008BD00BF91
:1043C000000C014030B1012809D1064BD868C0F378
:1043D00080007047034BD868C0F3C00070470020CE
:1043E000704700BF000C014038B500242546E0B2FC
:1043F000FFF7C1FF18B10123A3401D43EDB2013403
:10440000082CF4D1284638BD20B9034B9868C0F376
:10441000C0307047002070470008014010B9C9083B
:1044200004F02EBF704708B107F0C4BD07F0CABD45
:1044300062B6704772B6704718B9024B4FF480628B
:104440005A617047000C014018B9024B4FF480626A
:104450001A617047000C0140034B4FF4005208B141
:104460001A6170475A61704700100140074B9A88E3
:10447000C2F30722042A06D19A88D2B29D2A02D119
:10448000188980B270470020704700BF006C004060
:10449000034B4FF4804208B11A6170475A6170476C
:1044A0000010014038B5184B184C9A6812F480552A
:1044B00001D0206838BD03F055FF2A466060FF2117
:1044C000032000F057FA01220546FF21032000F0E7
:1044D00051FA40EA052010F002034FEA900018BF9D
:1044E0000123C204237203D5237A43F0020323720B
:1044F000830403D5237A43F004032372E36823EA99
:104500000000206038BD00BF001001406805002099
:104510005F4B70B59B68D90400F1B980FFF7C2FF0B
:104520005C494C690861A04234DD8B69051B9D42E2
:10453000594B0CDA1C68D1E908236C43121943EB80
:10454000E473C1E908238B6A1D448D6259E091F838
:104550002C6072070CD5CC681A68041B624326F0E5
:104560000406D317C1E908238C6281F82C6033E07C
:10457000CE681B68241A344404FB0334D1E90823B1
:10458000121B63EBE473C1E90823F6438B6A3544DD
:104590002B4411E035DA8B69221A9A423E4B0DDA30
:1045A0001D68041B5543D1E90823521B63EBE573D7
:1045B000C1E908238B6A23448B6222E091F82C50D6
:1045C0006A070ED51A6825F004054243D317C1E9DE
:1045D0000823886281F82C5000220023C1E90C23B3
:1045E0000FE0CA681D680132041B14446543D1E919
:1045F0000823521943EBE573C1E908238B6A1C4475
:104600008C628C6A8D6BCA6B651B85EAE576A6EBBE
:10461000E57696421F4B2ED95E681A6CB21A642A50
:1046200029D91E6442F2107675435A6495FBF2F262
:104630003C256A43DE689C63013692FBF6F29A647D
:1046400040F6B834002AB8BF5242A24201DDC82267
:1046500003E0B2F57A7F02DD6422DA6316E0322AE3
:1046600001DD0A22F9E70A2A01DD0522F5E7012A20
:104670000CDD0122F1E74C680A6C064BA21AB2F578
:10468000FA6F03D90122DA6300229A64486170BD8F
:1046900000100140680500200400002008B568B93A
:1046A000FFF736FF0649D1E90823D1E90C01121AB8
:1046B00063EB0103100A40EA036008BD002008BD57
:1046C0006805002038B50D46F8B9104CFFF720FFFB
:1046D000D4E90801E268002871F100034FEA0222E0
:1046E00002DA404261EB4101D3170BF00DF8C4E947
:1046F0000C23E9170B022A02D4E90C0143EA1563E3
:10470000121843EB0103C4E9082338BD68050020F3
:1047100010B9024B09011960704700BF0400002066
:1047200010B9024B83F82C10704700BF68050020B9
:10473000014B986C704700BF6805002010B9024B10
:10474000187A7047002070476805002038B5214B63
:10475000214A1B69214C5909090103F01F0311600B
:104760000320FE21002284F82C3000F003F94021C0
:104770000122032000F0FEF800210A46032000F089
:10478000F9F8002105460122032000F0F3F8082D76
:1047900005D140F6FF73E3604FF4006304E040F29C
:1047A000FF33E3604FF40073E72100220320A3618D
:1047B00000F0E0F800210122032000F0DBF8FFF711
:1047C00071FE60610002C117C4E90C01C4E908016F
:1047D00038BD00BFC80E002004000020680500207E
:1047E00008B5082003F062FE5E2805D9074B93F850
:1047F0004C2052B9012206E0082003F057FE54284D
:1048000003D8024B002283F84C2008BD6805002025
:10481000044B93F84C00013801288CBF0020012084
:10482000704700BF68050020044B93F84C00012836
:1048300006BF022283F84C20002070476805002044
:10484000002070472DE9F04F4FF4804089B00121DE
:1048500007F07EFD434C0120014607F06DFD032665
:104860004FF420434FF0180A204602A9ADF8083053
:104870008DF80BA04FF0040B8DF80A6007F0E5F9F6
:104880004FF48043204602A9ADF808308DF80A6045
:104890008DF80BB007F0D9F90823ADF81830324B7A
:1048A000002401254FF482794FF002084FF400777D
:1048B000184603A9ADF80C40ADF81040ADF81A4009
:1048C000ADF81C400193ADF80E90ADF81280ADF834
:1048D0001450ADF8167007F0E7FD019B2946184605
:1048E00007F068FE29464FF4805007F025FD284662
:1048F000214607F039FA8DF80BA0DFF874A0A02349
:10490000504602A9ADF808308DF80A6007F09DF90D
:104910004023504602A9ADF808308DF80A608DF8A2
:104920000BB007F092F9ADF80C40ADF81040ADF8BF
:104930001A40ADF81C400D4C1023204603A9ADF8D9
:104940001830ADF80E90ADF81280ADF81450ADF8F7
:10495000167007F0A9FD2046294607F02BFE09B086
:10496000BDE8F08F000C01400038004000300140ED
:104970000008014070B504460D461646032869D864
:10498000DFE800F00206090E4FF48052324B11E0CE
:104990001022324B02E0304B4FF400625A611CE0AF
:1049A0002F494FF400420B8823F002031B041B0C19
:1049B0000B802C4B5A612A48022107F07FFE002809
:1049C000F9D02748294607F025FE2548012107F0A0
:1049D00075FE0028F9D08EB92FE02348022107F098
:1049E0006DFE0028F9D02048294607F013FE1E4826
:1049F000012107F063FE0028F9D0ECE7032C29D849
:104A0000DFE804F002070A0F134B4FF480521A61DB
:104A10001BE01022114B02E00F4B4FF400621A61B1
:104A200011E0104B4FF400421A61A3F558431A8865
:104A300092B242F002021A8007E0032C0AD8DFE8A3
:104A400004F004020204084800E0054807F0E4FD11
:104A5000C0B270BD002070BD000C014000080140D4
:104A600000380040001001400030014037B5C54D0E
:104A7000A8786B782C4608B10422D8E2A52B00F068
:104A80002F8276D8852B00F01C8127D8072B00F0C9
:104A90004A810FD8032B00F0148105D8012B00F0B8
:104AA000E18040F2D580ECE0052B00F0258140F25A
:104AB00013812BE1812B00F0D58009D80D2B00F05C
:104AC0004E81802B00F0C4800C2B40F0AF8236E189
:104AD000832B00F0018140F26381D2E0952B00F03E
:104AE0007D811FD88C2B00F0708110D8872B00F0AF
:104AF0005E81C0F001818A2B40F098820020142151
:104B000001AA05F0E1FDEB788DF8063052E1932B18
:104B100000F0258100F213818D2B40F08782002068
:104B20001A213FE1A12B00F0BE8116D89A2B00F08C
:104B30006481A02B00F0B081992B40F0778201AA0C
:104B40000020182105F0C0FDEA789DF8053002F03C
:104B50000F0223F00F0313435BE1A32B00F0A981A5
:104B600000F2AE81D5F803100020C9B204F064FA57
:104B70005FE2B62B00F0258236D8AD2B00F0F9812C
:104B800015D8A92B00F0DA8105D8A72B00F0C88131
:104B900040F2B681CBE1AB2B00F0D68100F2DB8195
:104BA000D5F803100020C9B204F00EFB41E2B12B8E
:104BB00000F0F3810BD8AF2B00F0E18100F2E68129
:104BC000D5F80310002049B204F050FB31E2B32BBA
:104BD00000F0F081C0F0E781B52B40F02782D5F8D6
:104BE0000320694B9A6124E2C82B00F02A8114D873
:104BF000C12B00F0188108D8B82B00F0F981C0F063
:104C0000E981C02B00F08F8010E2C32B00F01481EB
:104C1000C0F00D81C72B79D008E2D42B00F01F81A2
:104C20000DD8D12B00F0EB81D22B00F0EE81CC2BF4
:104C300040F0FC81D5F80320534BDA81F9E1D62B03
:104C400000F01781C0F01081FE2B00F01781EDE11C
:104C500004F0A6FC20B9A178490101F0E0010BE0C5
:104C60000622E4E104F09CFC0028F9D1A178490176
:104C700041F0020101F0E201D4F8032005F08FFCBD
:104C8000D7E104F08DFC05460028E9D1A178D4F8DD
:104C90000320490141F0080101F0E80105F06DFC35
:104CA000A178D4F80320490141F0060101F0E601A2
:104CB0002846002AB8BF524205F05FFCA3780121C4
:104CC00017E004F06DFC0028CAD1A178490141F039
:104CD0000A0101F0EA0165E00621D4F80320002072
:104CE00005F04BFCA378D4F80310284A42F82310AF
:104CF0000021274AD1549CE1D4F80310002005F08C
:104D000056FDA378D4F80310224AEFE7224B012284
:104D10001A70E1781C4B5972204B1B78022B40F023
:104D20008881002061E11C4B01221A70E178164B4A
:104D300099721A4B1878002840F07B8155E101AA3E
:104D40000020142105F0C0FCD4F803209DF80530A4
:104D500012B143F0020311E023F002030EE001AAB6
:104D60000020142105F0B0FCD4F803209DF8053094
:104D700012B143F0010301E023F001038DF8053087
:104D800018E000BFC8090020C80E00204C0E00200B
:104D9000B8050020480A00202C0F00202F0F00200B
:104DA00000200421D4F8032005F0E7FB41E10020B6
:104DB0000E21F7E7A1780020490141F0140101F02C
:104DC000F40101AA05F0B4FB33E1E9789A4BD972FA
:104DD000C1F10801C9B204F0F5F82AE101AA1421D1
:104DE00005F072FCD5F803209DF8053012B143F0B0
:104DF0000403C3E723F00403C0E701AA002018213D
:104E000005F062FC9DF80530EA7803F00F0343EAF1
:104E10000213A1788DF80530490141F018010020F6
:104E200001F0F801CDE7EA78834B1A7201E1D5F879
:104E30000320814B1A60FCE0D5F803207E4B5A60BA
:104E4000F7E07E4B01221A707B4BD5F80320DA770E
:104E50007B4B1B78032B40F0EC80E978C5E0D5F85C
:104E60000320754B5A61E4E0D5F80320724B9A7722
:104E7000DFE0D5F80320704B9A83DAE0D5F80330F1
:104E8000052B6D4B05D86F4AD0781873FFF700FBE0
:104E9000CFE000221A73CCE0D5F803100020C9B28D
:104EA00004F09EF8C5E0D5F80310C9B204F0A4F8E8
:104EB000BFE0D5F803100020C9B204F0C7F8B8E08D
:104EC000002004F025F9D5F8031020B9A878C9B25C
:104ED00004F0D0F8ADE0A878C9B204F0F3F8A8E087
:104EE00004F016F9AB78D5F8031020B91846C9B20A
:104EF00004F0CAF89DE01846C9B204F0F7F898E04B
:104F0000002004F005F9D5F8031020B9A878C9B23B
:104F100004F0C4F88DE0A878C9B204F0DDF888E0A8
:104F2000D5F803100020C9B204F0C2F881E0D5F82A
:104F300003100020C9B204F033F97AE0D5F8031069
:104F4000C9B204F037F974E0D5F803100020C9B2F3
:104F500004F044F96DE0D5F803100020C9B204F064
:104F600047F9AA78384B03EBC203D5F803205A71EE
:104F70005FE0D5F80310C9B204F06EF959E0D5F836
:104F800003100020C9B204F0A1F952E0D5F80310D3
:104F90000020C9B204F0A4F94BE0D5F80310C9B25F
:104FA00004F0A8F945E0D5F803100020C9B204F0D8
:104FB000ABF93EE0D5F803100020C9B204F0B8F90F
:104FC00037E0D5F80300204B186090BB597904F006
:104FD0000FF92EE01C4BD5F803201A71184B1B78E3
:104FE000012B26D1174B0020D978FFF717FA20E0C4
:104FF000D5F803100020C9B204F032F819E00020FF
:10500000D5F80310FFF75EFB13E0D5F803200A4B39
:10501000E9781A61002001F01F01FFF781FBD5F844
:105020000310A8784911FFF773FB02E00322074B36
:105030001A7003B030BD00BFC80E00202C0F002036
:105040002F0F0020C80900205C0E00203C0A002021
:1050500073B5CD4ECD4CB0787378354610B104237E
:10506000237059E2A52B00F0ED8100F28E80842B95
:1050700000F0248138D8082B00F0328115D8032B9A
:1050800000F01F8105D8012B00F0128140F20D8144
:1050900014E1052B00F01C81C0F01881062B00F0F4
:1050A0001981072B00F0198124E20D2B00F02B81D0
:1050B0000BD80A2B00F04581C0F02D810B2B00F09E
:1050C0002F810C2B00F0158114E2812B00F0F08071
:1050D00003D8802B00F0E9800CE2822B00F03F81A6
:1050E000832B00F0F38005E2992B00F0438130D848
:1050F0008C2B00F03A8112D8862B00F0E980C0F0AA
:10510000E080872B00F02E818A2B40F0F381002075
:10511000142101AA05F0D8FA9DF80630E1E1932B9D
:1051200000F0F18005D88D2B40F0E48100201A2199
:10513000C9E0942B00F0DD80952B40F0DB8100204E
:10514000142101AA05F0C0FA9DF80530C3F38003CD
:10515000C7E1A02B00F05B810BD89B2B00F0E08017
:10516000C0F022819C2B00F0EC809D2B00F0B880D9
:10517000C0E1A22B00F05281C0F04C81A32B00F0C3
:105180005181A42B00F05281B4E1C02B00F0A58026
:1051900047D8AF2B00F0848121D8AA2B00F0728170
:1051A0000ED8A72B00F06681C0F05881A82B00F024
:1051B0006581A92B40F09E81002004F02DF87BE052
:1051C000AC2B00F06681C0F06081AD2B00F06481F3
:1051D000AE2B40F08F81002004F066F86CE0B42B19
:1051E00000F06D810ED8B12B00F06181C0F05B81C1
:1051F000B22B00F06081B32B40F07C81002004F0E2
:10520000E3F859E0B62B00F06081C0F05B81B72B6A
:1052100000F05E81B82B40F06D81002003F080FF2C
:105220004AE0CF2B00F0D9801FD8C52B00F0CD80ED
:105230000CD8C22B00F0C480C0F0BF80C32B00F09C
:10524000C180C42B40F05681514B3FE1C82B00F088
:10525000BE8002D8C72B3DD04CE1CC2B00F0BA80E9
:10526000CE2B40F047814B4B30E1D52B00F0C9806D
:105270000DD8D12B00F02F81C0F0C180D22B00F0CF
:105280002E81D42B40F03681434B5B6929E1D72B2B
:1052900000F02981C0F0B880DB2B00F02781FE2BC5
:1052A00040F028813C4B1B7B1BE10020014601E0C4
:1052B0000020022105F006FC60601DE100200821AD
:1052C00001E000200A2105F016FAF5E7334BFDE076
:1052D000334BFBE0304B5B7A03E12F4B9B7A00E1D1
:1052E000002005F0ECF9AB785B00184100F00103F9
:1052F000F7E00020142101AA05F0E6F99DF8053039
:10530000C3F34003EDE00020142101AA05F0DCF90D
:105310009DF8053020E0234B9B68C3F34013E0E089
:1053200001AA00207C2105F0CFF9AA7802235200BF
:1053300003FA02F29DF806301A420CBF0023012343
:10534000CFE001AA00207C2105F0BEF9AB789DF8E2
:1053500006205B0042FA03F303F00103C1E00020E2
:105360000421B0E700200E21ADE703F04DFEC0F1AF
:105370000800A1E7182101AA05F0A6F99DF805305B
:1053800003F00F03ADE000BFC80900203C0A002075
:10539000540E0020700E0020C80E00204C0E00207D
:1053A000480A0020000C01400020182101AA05F045
:1053B0008BF99DF805301B0993E0584B1B7A90E060
:1053C000564B83E0554B5B688BE0554B7EE0534B6F
:1053D000DB7F86E0514BDB8983E0524B60601A78BB
:1053E0000AB10122626000221A704F4B1A781AB17A
:1053F000626842F00202626000221A707CE04B4B4D
:105400005EE0464B9B7F6CE0444B9B8B69E003F076
:1054100003FE51E7002003F007FE4DE7002003F0F4
:105420006FFE49E7002003F073FE45E7002003F01C
:105430006FFE18B9B07803F07BFE3DE7B07803F05B
:1054400097FE39E703F064FEB37818B9184603F005
:1054500077FE31E7184603F09BFE2DE7002003F0AE
:1054600057FE18B9B07803F073FE25E7B07803F063
:1054700087FE21E7002003F073FE1DE7002003F004
:10548000C1FE19E703F0D0FE16E7002003F0D4FEBA
:1054900012E7274B5B7924E0002003F0FBFE0BE7CB
:1054A00003F06AFF08E7002003F06EFF04E7002026
:1054B00003F072FF00E7002003F076FFFCE61D4BCF
:1054C0001B780EE0154B9B690BE0194B1B6808E03D
:1054D000174B1B7905E00020FFF7E0F8ECE60F4BD7
:1054E0001B69636008E0FEF7DDFFE5E60020FFF7DB
:1054F00025F9E1E6032323700F4B1B7863B10F4BB3
:1055000062681A600E4B1AB91A6842F0080202E08B
:105510001A6822F008021A6002B070BDC80E00209E
:10552000EC0E0020C00E0020650E0020C10E0020F1
:105530005C0E00205A0E0020370A0020280A0020A6
:10554000D009002038B5B44A95781446022D00F0F1
:105550003281032D00F03681002D40F0B381537865
:105560004F2B00F0BD803BD8462B00F0918014D823
:10557000422B7BD009D8402B74D0412B40F0A08126
:10558000D178A64B0020197074E0442BA34A75D043
:105590007AD8E178042011716CE0492B00F08A8000
:1055A0000AD8472B7FD0482B40F08A81D3789B497B
:1055B000262001F8263FD3E04C2B00F087804D2BAE
:1055C00000F089804B2B40F07B81944CD1780320F4
:1055D000E17002F078FBE078BDE8384002F042BEAE
:1055E000572B00F0CB8013D8522B00F0A08006D8A8
:1055F000502B00F08880512B00F08A8060E1542B02
:1056000000F0A380C0F09A80552B00F0AB8057E1EA
:10561000832B00F0C1801AD8592B00F0B5805A2B8B
:1056200040F04E817D4DD378294601F8283F28204F
:10563000012202F0A7FB95F82800BDE8384010F0E1
:1056400001001ABF00200121014605F089BA852B0F
:1056500000F0AC80C0F0A580FF2B40F03181D27803
:105660006F4B31E140F2FF70D17803E0D1786B4BA2
:1056700001205970BDE8384002F025BBD4F8033052
:105680001C20D361674909E0E17805205171F1E7F9
:10569000D2F8033061490C2041F80C3F0422BDE8E8
:1056A000384002F06FBBD2F803305C49082041F863
:1056B000083FF3E7D278594B0AB9DA7503E05A4943
:1056C0000122DA754A601720D97DD3E7D178534B90
:1056D00002209970CEE7D178504B15205975C9E753
:1056E000D2F803104D4CC9B21920617602F0EBFAE2
:1056F000607E10F001001ABF284601210146BDE876
:10570000384005F01BBAD178444B16209975B1E7A3
:10571000424B1A7D1D4612F0010F04D0E378DB07DF
:1057200001D402F034FAE17814202975A2E7D2F806
:1057300003303A49202041F8203FAFE7D2F8033048
:105740003649102041F8103FA8E7D2F80330012B6A
:1057500000F2B880304B3149DB781A2001F81A3F4B
:1057600001229CE7D2F80330012B00F2AB802A4BD8
:105770002A49DB781B2001F81B3FF1E7D378274942
:10578000272001F8273FEBE7D2F8033023492420F4
:1057900021F8243F022282E7D2F80320234B5A60EB
:1057A00038BDD2F80320224B1A6038BDD2F803204E
:1057B0001E4B9A6038BD51781E4BD2F8032043F837
:1057C000212038BD5378272B62D01AD8022B48D01D
:1057D0000CD8002B3CD0012B72D1174BD2F80320F0
:1057E0005A6002F0BFFD114B186138BD1B2B41D030
:1057F0001C2B46D0092B63D1D2F803200E4BDA6064
:1058000038BD2B2B4DD019D8292BD2F803200A4BA9
:1058100043D044D85A6138BDC80900200800002090
:10582000360A0020240000203C0A0020B805002091
:10583000380A00204C0A0020F00E00202D2B3AD010
:1058400034D32E2B3CD1D2F80320204BDA6238BD62
:105850001E4BD2F803201A6002F084FD1C4BD86066
:1058600038BD1A4BD2F803209A6002F07BFD184B2A
:10587000586138BD0020D2F80310BDE8384005F06B
:1058800082B80020D2F80310BDE8384005F0A5B872
:10589000D2F803200D4B1A6138BD9A6138BDDA6128
:1058A00038BDD2F80320094B1A6238BDD2F8032064
:1058B000064B5A6238BDD2F80320044B9A6238BDB9
:1058C000032200E00422034B1A7038BDF00E0020C2
:1058D000B80500203C0A00202DE9F843044615468F
:1058E0000E4600294AD0002848D0814246D04FEACF
:1058F00042185FFA88F848F006073946002005F09C
:10590000E1F848F00C018146002005F0DBF8804604
:10591000204609F0BBFC0446304609F0B7FC0146BE
:10592000204609F0BFFD0646484609F0AFFC314667
:1059300009F0B8FD09F0C8FE0446404609F0A6FC8F
:10594000314609F0AFFD09F0BFFE002C08BF01246D
:105950000B49002814BF80464FF00108304609F07B
:105960008BFE18B12846414604F021FF2246002054
:10597000394604F014FE034B01225A55BDE8F88362
:105980000000A041B805002070B50C4D04462B5C0A
:105990009BB1C6B20A4B710141F0060153F82420B5
:1059A000002001F0E60104F0E8FD064B304653F814
:1059B000241004F0FCFE00232B5570BDB805002018
:1059C0004C0E0020480A00202DE9F341B94EBA4F91
:1059D0003378D6F803006422222B7B703A7078600B
:1059E00035463C4601F034815BD80F2B00F0AD8585
:1059F00026D8072B00F0C58111D8032B00F0D880E2
:105A000007D8012B00F0BD80022B00F0C58001F00B
:105A10009DBB052B00F0AD8140F2DF80ADE10B2B8B
:105A200000F0ED8405D8092B00F0A68340F27482C3
:105A3000A6E30D2B00F0168540F2FE8400F05DBD5C
:105A4000192B00F0D38614D8152B00F0328607D816
:105A5000132B00F0D185142B00F0098601F076BBE2
:105A6000172B964B00F0A88600F2B386D86101F0A0
:105A7000F0BB1E2B00F0D4840CD81B2B00F0D88672
:105A8000C0F0C5861C2B41F061838C4B00221A7636
:105A900001F0DFBB202B01F0348040F2F98701F0E8
:105AA00083B8812B01F05D8135D8412B01F047810E
:105AB00017D8252B01F0078107D8232B01F0CF80C1
:105AC000242B01F0D38001F041BB272B01F0298169
:105AD000C1F00281402B41F0398303F04AF801F014
:105AE000B8BB452B01F0348108D8432B01F02A8143
:105AF00001F22B8103F03FF801F0ABBB472B01F023
:105B00002D81C1F02881802B41F020836B4B002236
:105B10001A7601F09EBB882B01F0AD811BD8842B37
:105B200001F050810DD8822B01F02F81832B41F0A1
:105B30000D83624B002183F8441083F82C1101F08F
:105B400028B9862B01F05D8101F2CA815B4B0022EE
:105B50001A7601F07EBB8C2B01F01D8206D88A2BB1
:105B600001F0FD8141F2E38101F010BAF22B01F066
:105B70009D82FF2B01F0E0828D2B41F0E78201F046
:105B80002EBAB37853B903F00BFD002801F0E1827F
:105B90000623237001F05DBBB3781BB1042323708F
:105BA00001F057BB03F0FCFC002801F0F782EFE79F
:105BB000B578002DF2D1424B28461D70414B1D7027
:105BC00004F00CFC28462946022204F0ACFD2846CD
:105BD000082104F05DFD01F03CBB03F0E1FC00286E
:105BE000D6D1B378002B40F09980324B5B78032BF1
:105BF00000F2BB80DFE803F002296C960020FFF77B
:105C0000C3FEB1782F4B00245C542D4B2E4E5C54B8
:105C100001238B403278490122EA0303204601F038
:105C2000E001D5F80320337004F0B9FCA9782246CE
:105C3000204604F078FDAB78244901EB4312927FB3
:105C4000002A41F0D28201F004BB0020FFF79CFE45
:105C5000B3781C4A0026D654194A3046D6545B0104
:105C600043F0020101F0E20104F02CFFA9780123C6
:105C70008B40154FD5F803803A788044490122EAD9
:105C80000303304601F0E00142463B7004F087FC1C
:105C900030463246A97804F046FDA8780B4AC4F88D
:105CA000048002EB40139B7F002B41F0B78201F090
:105CB000D0BA00BFC80900203C0A0020B805002067
:105CC000C00E0020650E0020590E0020C80E0020D6
:105CD000D5F80330C54E142B20DCC54A002052F8FD
:105CE0002350FFF751FEB17801228A40C14B0024B6
:105CF0005C54C14B5C54C14B4901187801F0E00180
:105D000020EA02021A7020462A4604F048FC204687
:105D1000B178224604F007FD01F09BBA04232370FA
:105D200001F097BAD6F80320B14B002053F8226057
:105D3000FFF72AFEA97801228A40AE4B00245C546A
:105D4000AD4B5C54AD4B4901187801F0E00120EAFD
:105D500002021A702046324604F021FC2046A9783F
:105D6000224604F0E0FC01F074BA03233B7001F01A
:105D700070BAFEF77BFE01F06CBAFFF769F901F02B
:105D800068BAB078737800287FF408AF9A2B2AD8C5
:105D9000992B79D2822B65D00BD8062B54D003D8FF
:105DA000042B4BD0052B0AE0072B54D00C3B012BC6
:105DB00011E08C2B5BD00AD8832B3FD0862B40F090
:105DC000A78000200C2104F0A6FD01F042BA8D2B23
:105DD00054D0933B022B00F29B800020142104F04E
:105DE0009AFD01F036BAC82B6FD00DD8C12B57D011
:105DF00004D8B52B4DD0C02B2DD089E0C32B5DD05E
:105E000055D3C72B20D083E0D42B6CD00AD8CC2B11
:105E100062D0D22B7CD150207949042201F0B2FF0C
:105E200001F017BAD62B6CD064D3FE2B70D14C2066
:105E30007449012201F0A6FF01F00BBA00200621EF
:105E400004F069FD01F005BA6F4B4920597A01F061
:105E50003AFF01F0FEB96C4B4A20997A01F033FF0A
:105E600001F0F7B9042104F056FD01F0F2B94B201E
:105E70006649012201F086FF01F0EBB900201A21EA
:105E800004F049FD01F0E5B9182104F044FD01F0EA
:105E9000E0B958205E49042201F074FF01F0D9B93D
:105EA000594B4820197A01F00EFF01F0D2B9402079
:105EB0005849042201F066FF01F0CBB9442056494D
:105EC000042201F05FFF01F0C4B95F2053490122B1
:105ED00001F058FF01F0BDB94E205149022201F0F6
:105EE00051FF01F0B6B954204E49042201F04AFF97
:105EF00001F0AFB95E204C49012201F043FF01F0EF
:105F0000A8B95C204949022201F03CFF01F0A1B987
:105F10000323237001F09DB9A878344E6B780028D4
:105F20007FF43CAE9A2B46D8992B80F0EB80822BE5
:105F300000F0CC800ED8062B00F0BA8004D8042BD9
:105F400000F0A080052B0DE0072B00F0B8800C3B83
:105F5000012B28E08C2B00F0BE801FD8832B00F093
:105F60009180862B40F0048100200C2104F0B0FCCD
:105F7000AC780020610141F00C0101F0EC0104F06B
:105F8000BAFB2B4B2B4A43F82400A878002111546C
:105F900053F8201004F00BFC01F05BB98D2B00F0DE
:105FA000AC80933B022B00F2E3800020142104F02C
:105FB0008FFC01F04EB9C72B7AD03DD8C12B00F031
:105FC000AD8005D8B52B00F0A280C02B77D0CFE0F4
:105FD000C22B00F0AA80C32B40F0CA8044200E4997
:105FE000042201F062FF01F034B900BFC8090020AB
:105FF000D4090020650E0020C00E0020590E00209C
:10600000D80E0020D40E0020C80E0020D30E002091
:10601000E00E0020C80E0020CC0E0020E70E00206D
:10602000D60E0020DC0E0020E60E0020E40E00203C
:10603000480A0020B8050020D42B00F084800BD83B
:10604000C82B79D0CC2B40F093804E20AA49022255
:1060500001F02BFF01F0FDB8D62B00F0828079D340
:10606000FE2B40F08580A54C4C2004F10C01012250
:1060700001F01BFFB37804EB4314207BFEF708FA12
:1060800001F0E7B80020062104F022FCAC780020E3
:10609000610141F0060101F0E60104F02CFB984B90
:1060A000984A43F82400AB780021D15401F0D1B8CC
:1060B000492001F0E1FE914B587201F0CAB84A2024
:1060C00001F0DAFE8D4B987201F0C3B8042104F0A0
:1060D000FFFB01F0BEB8894C4B2004F10B010122FB
:1060E00001F0E3FEB07804EB4014E17AC1F108015D
:1060F000C9B202F067FF01F0ACB81A2104F0E8FB66
:1061000001F0A7B8182104F0E3FB01F0A2B8582071
:106110007D49042201F0C9FE01F09BB8482001F03E
:10612000ABFE764B187201F094B8402077490422F8
:1061300001F0BBFE01F08DB85F207549012201F02E
:10614000B4FE01F086B854207249042201F0ADFE7D
:1061500001F07FB85E207049012201F0A6FE01F037
:1061600078B85C206D49022201F09FFE01F071B801
:106170000323237001F06DB8FFF7E4F901F069B86B
:10618000B278674B022A00F0B180032A00F0D68073
:10619000002A40F01C815B78512B00F086802CD8BF
:1061A000472B70D014D8432B68D00AD8412B60D02D
:1061B00061D8402B40F0098140F2FF7001F05CFE95
:1061C000ECE0452B574A5CD040F28380D368FAE07C
:1061D0004C2B61D008D8492B5BD056D34B2B40F0C9
:1061E000F480504BDB78EEE04F2B58D05AD84D2B33
:1061F00040F0EB804B4B5B7DE5E0802B66D013D805
:10620000552B59D005D8532B464A51D052D8136A32
:10621000D9E0592B53D05A2B54D0572B40F0D5806E
:10622000404B93F82730CEE0842B56D008D8822BF1
:10623000344A4ED04FD8137E1E1F73427341C2E0C2
:10624000F02B4CD00DD8852B40F0BF802D4A36491D
:1062500093684B4303F540533933936023F0004375
:10626000B1E0FE2B3BD0FF2B40F0AF802F4B1B78D3
:1062700038E02C4B34E02B4B5B78A4E0294B1B79A6
:10628000A1E053799FE0274B83E0264B93F826301B
:1062900099E0244BDB7D25E0224B9B7893E0214B5A
:1062A0005B7E90E01F4B9B7D8DE01E4B1B7D8AE04B
:1062B000136988E0937E86E01A4BDB7E83E0194BFE
:1062C0009B8C80E0174B93F828307CE00D4B1B7EB5
:1062D00079E0D36977E0536875E0154B56E0154BCC
:1062E0001B7870E0003318BF01236CE05A78124B22
:1062F00053F8223067E000BFD60E0020C80E002001
:106300004C0E0020B8050020E00E0020C80E002032
:10631000E70E0020DC0E0020E60E0020E40E002038
:10632000C8090020080000206D4EC641360A002032
:10633000380A0020240F00204C0A00205B78272B0D
:1063400032D011D8022B23D005D8F3B1012B3CD188
:106350009F4B5B6837E01B2B1DD01C2B20D0092BDB
:1063600033D19B4BDB682EE02B2B24D005D8292B77
:10637000974B1CD01DD85B6925E02D2B21D01DD358
:106380002E2B22D1924BDB6A1DE0914B1B681AE049
:106390008F4B9B6817E0002004F049FB606018E019
:1063A000002004F059FBF9E7894B1B690BE09B695E
:1063B00009E0DB6907E0864B1B6A04E0844B5B6AFB
:1063C00001E0834B9B6A636003E0032300E0042346
:1063D0002370804B1B78002B00F03B877E4B62685C
:1063E0001A607E4B2AB91A6842F008021A6000F05F
:1063F00030BF1A6822F008021A6000F02ABFB37892
:10640000022B15D17378372B0ED8754903F5A77079
:10641000800001EB8301042201F0B4FC00F019BFFD
:106420007378142B40F203830323237000F011BF11
:1064300004233B7000F00DBFB378022B0ED1694BE3
:106440005B78372BF0D8664903F5A770800001EB25
:106450008301042201F029FD00F0FBBE04233B7000
:1064600000F0F7BEB378002B7FF498AB6B785D4EED
:10647000012B21D002D3022B23D03AE003F090F875
:1064800000287FF485ABB07803F0A0FFB17839B96C
:10649000554B01221A70554B00221A7000F0D9BEDC
:1064A000534A937F002B00F0D48602EB4112927F77
:1064B0009A4240F0CE86EBE7002003F08FFF00F019
:1064C000C8BE002003F092FF424B78601B78002B7F
:1064D00000F0BF86404B1860404B1A6820B942F06C
:1064E00008021A6000F0B5BE22F008021A6000F03F
:1064F000B0BE03233B7000F0ACBEB37813B1022BE7
:1065000004D01EE0FDF7A8FF00F0A3BE354B5B787A
:10651000072B0AD820B91846FDF704FF00F099BEF2
:106520001846FDF70BFF00F094BEFF2B7FF47CAF05
:10653000451C0ABF284BC0B21878FDF70BFF00F0CE
:1065400088BE04233B7000F084BEB378012B23D0B7
:1065500005D3022B24D17078FDF734FF0DE070785D
:10656000082802D8FDF707FF07E00A2801D1002319
:106570000BE00B2803D1FEF763F9606012E00C28F2
:1065800005D11C4B9B68C3F3401363600AE0FF28EE
:1065900008D1FDF729FFF0E7707801F087FFECE7FD
:1065A00004233B700B4B1B78002B00F052860A4BE8
:1065B00062681A60094B2AB91A6842F008021A6028
:1065C00000F047BE1A6822F008021A6000F041BECF
:1065D000F00E0020370A0020280A0020D0090020F1
:1065E0004C0A0020C8090020B8050020650E0020D4
:1065F000C80E0020000C01407278944B092A27D85D
:10660000DFE802F005080B0E12181B1E21251A6880
:1066100010441CE01A68101A19E01A68504316E07A
:106620001A6892FBF0F012E01A6892FBF0F100FB9E
:1066300011200CE01A68104009E01A68104306E0C7
:106640001A68504003E01A68D2431A6000E01860EC
:106650001A687F4B2AB91A6842F008021A6000F0E3
:10666000F8BD1A6822F008021A6000F0F2BD774BFC
:106670001A68774B8242196804DD21F0030141F06A
:10668000040108E00BBF21F0060121F0050141F0F3
:10669000010141F0020119602AB91A6842F00802AA
:1066A0001A6000F0D6BD1A6822F008021A6000F0E5
:1066B000D0BD73780C2B00F2CC85DFE803F0071017
:1066C00019222B343E475059626B7400604B1B6893
:1066D0001C0740F1BE855F4BD86100F0BABD5C4B32
:1066E0001B68190700F1B5855A4BD86100F0B1BDA0
:1066F000574B1B68DA0740F1AC85564BD86100F068
:10670000A8BD534B1B68DB0700F1A385514BD86133
:1067100000F09FBD4E4B1B685F0740F19A854D4BC3
:10672000D86100F096BD4A4B1B6813F0050F00F0CE
:106730009085484BD86100F08CBD454B1B689E0787
:1067400040F18785434BD86100F083BD404B1B6807
:106750009D0700F07E853F4BD86100F07ABD3C4B31
:106760001B68DC0640F175853A4BD86100F071BDBD
:10677000374B1B68990640F16C85364BD86100F0A9
:1067800068BD334B1B685A0640F16385314BD861B5
:1067900000F05FBD2E4B1B681B0640F15A852D4B48
:1067A000D86100F056BD2A4B1B68DF0540F15185CA
:1067B000284BD86100F04DBD1A6A072A00F24985BE
:1067C000511C1962D96903EB82025162D86100F051
:1067D00040BD1B6A1F4A002B00F03B85013B136242
:1067E00002EB83035B6AD36100F033BD73782E2B19
:1067F00004D8194A0121D15400F02BBDFF2B7FF49E
:1068000013AE144B012283F8442000F022BD7378AC
:106810002E2B04D8104A0021D15400F01ABDFF2BB2
:106820007FF402AE0B4B002283F8442000F011BD30
:10683000084C94F84530CBB9461C4FF00A030DD1F3
:10684000024A10684343A3640AE000BF280A0020FC
:10685000D0090020B8050020360F00205843A0645E
:1068600001F080FD0123E06484F845306B78042B4F
:1068700000F2EF84DFE803F0034372A7190001F090
:1068800071FDE26CA16C801A80EAE072A2EBE0720A
:106890008A42AE4B04D9002283F8452000F0D9BCCF
:1068A000DA69013ADA6100F0D4BCA87803F09EFD01
:1068B00040B9A74B84F845001A6822F010021A600C
:1068C00000F0C7BCA36CA14DA3B101F04BFDEB6C74
:1068D000AA6CC01A80EAE073A3EBE073934209D973
:1068E000002385F845309A4B1A6842F010021A606E
:1068F00000F0AFBCE369013BE36100F0AABC0020FB
:1069000003F0DDFEAB785B00184110F0010609D002
:10691000002384F845308E4B1A6822F010021A606A
:1069200000F097BCA36C894D9BB101F01BFDEB6C93
:10693000AA6CC01A80EAE073A3EBE073934208D913
:10694000834B85F845601A6842F010021A6000F027
:1069500080BCE369013BE36100F07BBC6A46002038
:106960007C2103F0B1FEAA780223520003FA02F25E
:106970009DF8023012EA030709D0002384F845305D
:10698000734B1A6822F010021A6000F062BCA16C0E
:106990006E4D99B101F0E6FCE96CAE6C401A80EAEC
:1069A000E071A1EBE071B14208D9694B85F84570FF
:1069B0001A6842F010021A6000F04BBCE369013B18
:1069C000E36100F046BC6A4600207C2103F07CFEB7
:1069D000AB789DF802205B0042FA03F313F0010646
:1069E00009D0002384F84530594B1A6822F0100270
:1069F0001A6000F02EBCA26C544D9AB101F0B2FCAA
:106A0000EA6CA96C801A80EAE072A2EBE0728A421A
:106A100008D94F4B85F845601A6842F010021A6099
:106A200000F017BCE369013BE36100F012BCB278EF
:106A30009AB9484A4849927E41F82300002A00F05A
:106A40000884002B00F0058403F28510800001EB20
:106A50008301042201F096F9FBE3FF2A7FF49EA84C
:106A600063B94FF4C3643D492046214404220434F1
:106A700001F088F9B4F5CD6FF5D1EAE3364903F2B8
:106A80008510800001EB8301042201F07BF9E0E333
:106A90007378142B3FF6C8AC314A9278B2B92E4ABB
:106AA00052F823202F4B7A601B78002B00F0D18303
:106AB0002D4B1A60264B22B91A6842F008021A6060
:106AC000C7E31A6822F008021A60C2E3FF2A7FF4C3
:106AD00065A863B94FF4C3642049204621440422C9
:106AE000043401F0E2F9B4F5CD6FF5D1B1E31A4900
:106AF00003F28510800001EB8301042201F0D5F937
:106B0000A7E37678142E3FF68FACA878144F0106D1
:106B10002CD5C20706D50020022103F0D3FF0E4B6F
:106B200043F826000B4B9B7E002B00F092836B7882
:106B3000002B00F08E83084903F28510800001EBE2
:106B40008301042201F01EF983E300BFB805002091
:106B5000D009002008000020D4090020C003002034
:106B6000C8090020370A0020280A002000287FF4E6
:106B700015A8022103F0A6FF994B9A4A9B7E42F882
:106B80002600002B00F065837B78002B00F06183EA
:106B9000B97803F285100844194402EB81018000A2
:106BA000042201F0EFF854E372788F4B0A2A42D89E
:106BB000DFE802F0060B11161C24292E33383C00A6
:106BC0008A491A6809680A4403E088491A6809680A
:106BD000521A1A602FE085491A6809684A43F8E793
:106BE00082491A68096892FBF1F2F2E77F4A196854
:106BF000126891FBF2F002FB1012EAE77B4A11687F
:106C00001A680A40E5E7794A11681A680A43E0E71A
:106C1000764A11681A684A40DBE7744A1168C9432A
:106C2000116008E01A6871490A6004E06F4A186848
:106C30001168106019601A686D4B22B91A6842F029
:106C400008021A6005E31A6822F008021A6000E3DD
:106C5000654B1B68C6F80330FDF708FFF9E2624B8D
:106C60001B68C6F80330FEF76DFCF2E27378052B63
:106C700000F2EF82DFE803F003090F151B215C4BE4
:106C80001A6802F00F021A60E3E2594B1A6822F008
:106C900010021A60DDE2564B1A6822F020021A60D8
:106CA000D7E2534B1A6822F040021A60D1E2504BEF
:106CB0001A6822F080021A60CBE24D4B1A6822F467
:106CC00080721A60C5E273782E2B3FF6ADAB494A4D
:106CD00002EB83031865BCE2464B4349D3F80C2111
:106CE0000A60D3F8102141490A60D3F814214049C1
:106CF000DA61D3F818210A60D3F81C213E4983F8E1
:106D00004520D3F82021DA64D3F824219A6493F83B
:106D10002821885C08B101208854002283F82C21A6
:106D200097E2B378002B7EF439AF7378142B3FF6DB
:106D30007BAB2D4A11682B4A42F8231089E201F0FF
:106D400019FF86E201F018FF83E201F027FF80E2DD
:106D500001F025FF7DE201F023FF7AE201F021FF3F
:106D600077E2737813B1012B04D00BE0214B0122A1
:106D70001A766EE2B0F5006FBEF410AF1D4A1376BE
:106D8000D06166E203233B7063E21A4B02221A765B
:106D90005FE2184A4FF0FF3002F1500343F8210040
:106DA00015480023435401312F29F2D11376D361C2
:106DB000136282F845300C4A13600C4A13600C4A87
:106DC000136046E2064B1B7D9B0717D4B0F5006F9E
:106DD000BEF4E4AE074B04221A76C3F8300138E261
:106DE00008000020D4090020280A0020440A0020BE
:106DF000D0090020B8050020360F002008233B7082
:106E000027E2994B01221A70984B994C9A78B0F569
:106E1000006F227025D21B7D13F0010521D1694638
:106E200000F074FE9DF80030257263709DF801300B
:106E3000A3709DF80230E3709DF8063023719DF831
:106E4000053063719DF80430A3719DF80330E37140
:106E50000123E15C227A01330A44082B2272F8D123
:106E6000F7E101230021E1540133082B804AF9D1D5
:106E700013781372EDE17378012B1DD00AD3022B26
:106E80002BD1794B01221A70784B794A9B78137079
:106E9000002319E0744B01221A70744B744A9B78DA
:106EA0001370744B186800230133C11811F8011CCA
:106EB000082BD154F8D1CCE10422FA717B719D22C8
:106EC0002423BA713B71C4E16B490133194411F8B1
:106ED000091C082BD154F7D1BBE103233B70B8E167
:106EE0007378032B00F2B581DFE803F0020E191D61
:106EF000624B1A7EFA7193F84520D3F83031BA719B
:106F00001A0A7A713B71A4E15C4B1A7EFA7193F80C
:106F10004520DB69BA711A0A7A713B7199E1584BC5
:106F20001B687B6095E1574B1B687B6091E1737830
:106F3000002B40F08E81544B9978002940F08981D4
:106F400040F2D243984240F0848140F2FF7000F05A
:106F5000BAFE00F01CFE0120FDF765FA79E17278B7
:106F60004A4B02B101221A70EA78494B1A70434B1E
:106F700093F83411474B1970474900230B70474968
:106F80000B70474B19780A431A7062E13B4B0122A0
:106F900083F835215DE1757815B1012D0FD01BE027
:106FA000042240F2FB70694600F07FFF009BD6F898
:106FB00003209A4206BF01237B607D6049E1B378DC
:106FC0002A2B06D140F2FB703649042200F0DAFE8B
:106FD0003FE103233B703CE103233B7039E17378CD
:106FE000032B3DD8DFE803F008022E39234A0023A3
:106FF000D2F83811154610E0204BD3F83821092A71
:1070000007D8511CC3F8381103EB8203C3F83C01C5
:107010001FE109233B701CE101338B4200F0198111
:10702000214A9E0052F823408442F5D13244481E42
:10703000834204D25068013342F8040BF7E7C5F8E5
:10704000380106E10D4A0023C2F83831164A002102
:1070500099500433282BF9D1FBE00A237B60F8E038
:1070600003233B70F5E000BF2C0A0020080000203D
:107070002D0A00200000002000400008B805002074
:10708000280A0020440A0020C8090020580E0020C9
:107090006C0E00202E0F0020660E0020650F0020D1
:1070A000590E0020CB090020F40600207378812BB4
:1070B00040F0CF80B278684B922A40F0CA809A792B
:1070C000A32A40F0C6805A79B42A40F0C2801A79C7
:1070D000C52A40F0BE80DB78D62B40F0BA805F4BEB
:1070E0004FF480621A6101F0E3FC01F03BF90446C1
:1070F00001F038F9001B0028B8BF4042B0F57A7F94
:10710000F6DBFDF797F904F06FFE002005F040FB79
:107110000021534804F041FA514804F0A3F95148C2
:1071200004F002F804F07EFA4FF0804005F086FB90
:107130000020FDF778F98CE040F2D243984240F00D
:107140008880494B012283F8642182E00223237066
:107150007FE0B37843B1454A02EB43139B7F002B9A
:1071600077D0927F9A4274D13F4B01221A70404BE4
:1071700000241C703F4B2046214602221C7003F065
:10718000D2FA2046062140F2FF7203F0F6F92046BB
:107190000821D5F8032003F0F0F95AE02E4B9B7834
:1071A00043B1324A02EB43139B7F002B51D0927FB5
:1071B0009A424ED12C4B01221A702D4B00241C7088
:1071C0002C4B2046214602221C7003F0ACFA2046CC
:1071D000062140F2FF7203F0D0F9D5F803202046D3
:1071E0000821524203F0C9F933E0002B31D08B7FE4
:1071F00093422ED12046FEF7C7FB3378204623F07A
:1072000001033370144B2146D3F8032003F0C7F970
:1072100020462146224603F086FA1AE0C8B1927F42
:107220009A4216D1FEF7B0FB0221304603F04AFC29
:10723000094B3146D3F803203B78024423F0010385
:1072400030463B7003F0ABF930463146324603F02E
:107250006AFA02B0BDE8F081C8090020000C0140C4
:107260000800024000240140B8050020C80E00209C
:10727000C00E0020650E00203749002370B50B605A
:107280003649374A0B603749D36113620B6082F885
:10729000453082F8443082F82C311546324A4FF09E
:1072A000FF3142F82310314A0024D45401332F2BEC
:1072B000F4D10621204603F005FC2D4B0C2118606B
:1072C000204603F0FFFB2B4E2B4BF17A1860C1F1E7
:1072D00008012046C9B201F075FE307BFDF7D8F8F1
:1072E000264B0022E2500434B4F5806FF8D1244ECE
:1072F000B37E13B9F37E6BB118E04FF4C364214938
:10730000204621440422043400F0CFFDB4F5CD6FB3
:10731000F5D1EFE74FF4A7641B492046214404222E
:10732000043400F0C2FDB4F5C36FF5D1337903F036
:10733000EF02012A01D0212B01D1012300E000231B
:1073400085F86531737D23B1FDF762FA08B1012339
:1073500000E000232B7670BD280A0020440A00209C
:10736000B8050020D009002008060020360F0020B4
:107370004C0E0020C80E0020480A00204C0A0020B5
:1073800008000020C003002014050020F7B50F4EB0
:107390000F4CC6F803300F4B86460F46B2700022E2
:1073A00094E803001A708DE8030086F800E0777017
:1073B000FEF70AFB21786368074A82F866119DE8A8
:1073C000030084E80300184603B0F0BDC80900209C
:1073D0003C0A0020370A0020B8050020014B93F832
:1073E00066017047B8050020F7B51F4E0246537876
:1073F0000C4696E803008DE803001C4900270B703B
:1074000093786D464B70D3788B7013798B71537969
:107410004B7193790B71D379CB70154B1F70FEF7BD
:10742000D3FA144B1978334671B9217032786170F0
:10743000A2707278E270F2792271B2796271727917
:10744000A2713279E27109E0012907D13A460A496D
:1074500011444978A1540132082AF8D195E8030073
:1074600083E8030003B0F0BD3C0A0020C8090020F7
:10747000370A00202C0A00202D0A00202DE9F043B5
:107480007E4B89B01B787E4C13B994F8673163B199
:107490007C4B1B78062B08D00A2B06D003F0EF0399
:1074A0000F2B1CBF002384F8343194F83431744A14
:1074B000032B754E2AD192F865511DBB33788BB9D9
:1074C000724F734DB87897F801802A7880449044C1
:1074D0006A789044EA799044AA7990446A79904411
:1074E0002A7920E0012B40F095806A4B585D0135E8
:1074F00000F086FE092DF8D18CE0072B6AD192F8B6
:10750000653173B3624803F091FD83E0042BF4D13D
:107510005E4F5F4DB87897F80180002301226B70B1
:107520002A706B608044904400F06AFE787800F026
:1075300067FE287800F064FE687800F061FEE87964
:1075400000F05EFEA87900F05BFE687900F058FE5E
:107550005FFA88F8287900F053FE404600F050FEAC
:1075600058E032782ABB494B93F802C093F8018067
:10757000474B8DF808C01F785D78C444D8798DF8E2
:107580000A70674499798DF80B503D445A798DF80B
:107590000C0028441B798DF80D1001448DF80E2045
:1075A0000A448DF80F3013448DF809808DF810309F
:1075B00008E0012A06D1374A995C02AA995401339E
:1075C000092BF8D1344B1B7823B302A8092101F011
:1075D000A3FA1FE0082B1DD12D4A00230120537070
:1075E00010705360294A8DF80A00917852788DF80E
:1075F00008108DF809200A4402448DF80B308DF8EC
:107600000C308DF80D308DF80E308DF80F308DF870
:107610001020D7E7214B1A789846002A6BD0204BD0
:10762000204D1B78032B02D0072B3DD05FE0174F76
:107630002A78B87897F80190814409F10A099144B1
:1076400000F0DEFD787800F0DBFD802000F0D8FD52
:107650008A2000F0D5FD002000F0D2FD002000F0CF
:10766000CFFD002000F0CCFD5FFA89F9287800F00A
:10767000C7FD484600F0C4FD39E000BF360A0020CF
:10768000B8050020C80900202C0A002008000020AE
:107690003C0A00202D0A0020500E0020650F00201B
:1076A0002E0F0020660E0020964B2A789878597885
:1076B00080238DF816308A238DF8173000238DF83B
:1076C00018308DF819308DF81A308F4B8DF8151051
:1076D00001440A311B788DF81B200A448DF81400F0
:1076E0008DF81C201BB105A8092101F015FA002313
:1076F0002B7088F80030002384F83431337084F81C
:10770000673194F8643113B10120FCF78CFE94F8D2
:1077100035217E4B52B193F86521D2F1010238BF79
:10772000002283F86521002283F8352194F8655101
:10773000002D71D10DF1070000F07CFD00286BD009
:1077400000F096FD10B1714B83F8685194F8681100
:107750009DF807004A1CD2B22144092A6B4B84F8D9
:10776000682181F8690140F0DD80002283F86821FA
:10777000644A93F869315178994207D092F82710FA
:10778000002900F0CF808B4240F0CC8092F8272077
:107790009A4204BF012384F8673100231A465B4DE7
:1077A00005F26911595C01330A44082BD2B2F6D1B3
:1077B00095F8713193422BD1554B95F86A211A7087
:1077C00095F86B215A7095F86C219A7095F86D2197
:1077D0009A7195F86E215A7195F86F211A7195F882
:1077E0007021DA7000F0BEFD4A4B4B4A1860297ECA
:1077F00000231370032285F834214A1E012A85F8DC
:107800006831464A02D9052918BF0123137089E05F
:10781000042385F8343185E094F865313B4D7BB124
:107820003B4803F0B6FA58B100F09CFD394B3A4A98
:10783000186000231370032285F834212A7E3AE071
:1078400094F86561002E44D12F4B1B78002B40D05B
:1078500005AD284601F04AF900283AD033463246B1
:10786000E95C01330A44082BD2B2F9D19DF81C100F
:1078700091422BD1264B9DF815201A709DF81620A9
:107880005A709DF817209A709DF818209A719DF8EB
:1078900019205A719DF81A201A719DF81B20DA7070
:1078A00000F060FD1B4B1C4A186000231370072278
:1078B00084F83421227E511E01291946174B03D921
:1078C000052A01D001221BE019702BE084F8343125
:1078D00028E0237E0D4D013B012B23D8EB69B3F546
:1078E000006F1DD2FCF794FFD0B1E8690849431C32
:1078F000EB6100F00BF9092385F83431074B0122C5
:107900001A700FE008000020500E0020B80500207B
:10791000C8090020280F00202D0F0020370A002062
:1079200000232376237E714D042B04D1704E3278D0
:10793000170640F1AD8094F8343113F0FB0F05D0F9
:10794000082B03D0062B01D0FEF73EF894F8343113
:10795000092B79D100F006FD644A664DD2682B6888
:10796000801A80EAE072A2EBE0729A4208D9624B78
:107970001A78012A04BF02221A7000F0F3FCE060BA
:1079800000F0F0FC23696A68C01A80EAE073A3EB98
:10799000E073934208D9584B5A78012A04BF022257
:1079A0005A7000F0DFFC206100F0DCFC6369AA681B
:1079B000C01A80EAE073A3EBE073934208D94E4B00
:1079C0009A78012A04BF02229A7000F0CBFC606111
:1079D00094F84430002B37D0444B93F82C21002AE4
:1079E00032D145498B5C022B2BD1404B03F1500027
:1079F00050F82200451C22D0404983F8282109680C
:107A00000022C3F80C113E490968C3F81011D96966
:107A1000D861C3F814113B490968C3F8181193F8E9
:107A2000451083F84520C3F81C11D96C0122C3F816
:107A30002011996C83F82C21C3F8241104E0002351
:107A40008B5401322F2ACCD194F83411274B0929B9
:107A500004D11A7E022A04BF05221A76D4F83821EE
:107A6000224B002A3ED009293CD1197E012939D167
:107A7000D86900231D4901F59E7454F82340A042A3
:107A800002D105230B762DE001339342F2D129E098
:107A900095F8343113F0FB0F24D0082B22D0062B9D
:107AA00020D0D5F83001184CD6F80330B0F5006F6F
:107AB0006270636012D2314600F03BF9D5F83001B4
:107AC000314600F0A8F830B1D5F830310133C5F8AF
:107AD0003031652300E00723237003E00723237080
:107AE00000232B7609B0BDE8F08300BFB805002065
:107AF000C8090020F00E0020360F0020280A0020C0
:107B0000440A0020D00900203C0A0020C0EBC0003D
:107B100038B500F5006500200C4602460321FCF74D
:107B200029FF0020C5F307210246FCF723FF0020B0
:107B3000E9B20246FCF71EFF002001460246FCF7B0
:107B400019FF2070002001460246FCF713FF607009
:107B5000002001460246FCF70DFFA0700020014600
:107B60000246FCF707FFE070002001460246FCF7E2
:107B700001FF2071002001460246FCF7FBFE607108
:107B8000002001460122FCF7F5FEA07138BD38B592
:107B90004FF40064002006210122FCF7EBFE0020D8
:107BA00005210246FCF7E6FE002001460122FCF713
:107BB000E1FE8307F3D5002002210246FCF7DAFE3E
:107BC0000020C4F307210246FCF7D4FE0020E1B2F6
:107BD0000246FCF7CFFE0025B5F13F0EDEF10002B4
:107BE0004FF0000052EB0E0201460135FCF7C2FED9
:107BF000402DF1D1002005210246FCF7BBFE0020FC
:107C000001460122FCF7B6FEC307F3D44034B4F5B5
:107C1000804FBFD138BDF7B5C0EBC00000F500659F
:107C200000200C4602460321FCF7A4FE0020C5F309
:107C300007210246FCF79EFE0020E9B20246FCF74F
:107C400099FE002001460246FCF794FE07460020FC
:107C500001460246FCF78EFE06460020014602461B
:107C6000FCF788FE0546002001460246FCF782FE2E
:107C70008DF80300002001460246FCF77BFE8DF8DC
:107C80000400002001460246FCF774FE8DF8050052
:107C9000002001460122FCF76DFE23788DF80600D6
:107CA000BB420DD16378B3420AD1A378AB4207D16E
:107CB000DDF80300D4F80330C31A5842584100E0FD
:107CC000002003B0F0BD38B5012204460D46002067
:107CD0000621FCF74FFE002005210246FCF74AFE74
:107CE000002001220146FCF745FE8207F3D5002063
:107CF00002210246FCF73EFE0020C4F307210246A3
:107D0000FCF738FE0020E1B20246FCF733FE00200B
:107D100029460122FCF72EFE002005210246FCF731
:107D200029FE002001460122FCF724FEC307F3D4FC
:107D300038BD38B5C0EBC0050C4605F500600978C4
:107D4000FFF7C1FF05F601006178FFF7BCFF05F6FC
:107D50000200A178FFF7B7FF05F60300E178FFF70F
:107D6000B2FF05F604002179FFF7ADFF05F6050027
:107D70006179FFF7A8FF05F60600A179BDE8384054
:107D8000FFF7A1BF2DE9F04104460F46164600203B
:107D900006210122FCF7EEFD002005210246FCF73A
:107DA000E9FD002001460122FCF7E4FD8507F3D53B
:107DB000002002210246FCF7DDFD0020C4F307216C
:107DC0000246FCF7D7FD0020E1B20246FCF7D2FDE7
:107DD0000025B54242D0013414F03F08795D04D04B
:107DE000721EA81A4242424100E001220020FCF724
:107DF000C1FDB8F1000F2FD1731E9D422CD200207F
:107E000005210246FCF7B6FD002001460122FCF7E1
:107E1000B1FD10F00100F2D106210122FCF7AAFD0C
:107E2000002005210246FCF7A5FD002001220146A5
:107E3000FCF7A0FD8207F3D5002002210246FCF7E3
:107E400099FD0020C4F307210246FCF793FD0020B2
:107E5000E1B20246FCF78EFD0135BAE700200521AC
:107E60000246FCF787FD002001460122FCF782FD57
:107E7000C307F3D4BDE8F08110B504460020032108
:107E80000246FCF777FD0020C4F307210246FCF709
:107E900071FD0020E1B20246FCF76CFDBDE8104028
:107EA000002001460122FCF765BD70B504460020A4
:107EB0000E46154603210246FCF75CFD0020C4F384
:107EC00007210246FCF756FD0020E1B20246FCF70E
:107ED00051FD0024AC420AD06A1EA31A00205A4267
:107EE00001465A41FCF746FD30550134F2E770BDBA
:107EF00037B5002005210246FCF73CFD0020014675
:107F00000122FCF737FD10F07104F2D100F02AFADB
:107F1000054600F027FA401B0028B8BF4042B0F5E4
:107F2000FA6F09DA4CB940F2FF70FFF7A5FFB0F124
:107F300042035C425C41ECE714B1224B1B78ABB3CB
:107F400040F2FF700021FFF7BEFEFFF720FE002089
:107F50001D494022FFF716FF4FF480701B49B422E1
:107F6000FFF710FF40201A492022FFF70BFF0023E4
:107F700001934FF4C364204601A904220434FFF79F
:107F800001FFB4F5FF6FF6D1002301934FF4A7640E
:107F9000204601A904220434FFF7F4FEB4F5C36FB0
:107FA000F6D140F2FF704221FFF78DFE0020064916
:107FB0004022FFF77AFF402006492022FFF775FF95
:107FC00003B030BD740E0020080000202405010815
:107FD00004050108C80E002030B5054687B0524898
:107FE00005F018F94FF48040012104F0A5F90420B0
:107FF000002103F0B9FE03238DF8063018230DEBA2
:1080000003048DF807304FF4007324F8143D4748FB
:10801000214603F01AFE48238DF8073043484FF4F9
:1080200080632146ADF8043003F00FFE02A805F08E
:108030007FF90B2D25D8DFE805F02406090C0F1277
:1080400015181B1E20224FF461531CE04FF4964379
:1080500019E04FF4E14316E04FF4164313E04FF4F8
:10806000614310E04FF496330DE04FF4E1330AE042
:108070004FF4613307E02E4B05E02E4B03E02E4B0F
:1080800001E04FF416530293029B02A95B082648B5
:10809000029305F009F92523002401258DF800300D
:1080A000684607238DF801308DF802408DF80350A3
:1080B00003F0D6FE1C4840F2FF3105F021FA2246BB
:1080C0001948282105F061F92A46174840F227711E
:1080D00005F05BF92A46144840F2266105F055F98F
:1080E0002A46114840F2255105F04FF922460E4824
:1080F00040F2244105F049F922460B4840F646017A
:1081000005F043F92246084840F66A1105F03DF9AA
:1081100022460548602105F038F90348294605F054
:1081200028F907B030BD00BF003801400008014009
:1081300090D0030020A1070040420F00684620F0C5
:1081400007018D46294919B50B889C061AD5284B7D
:10815000DB68980701D58B8814E0264B1A685868AD
:108160000132202A08BF0022824205D01C6888887C
:108170001919C0B208721A601F4A0A2111609A6A5E
:108180001E4B1A60194803881A061BD51B4B1A6828
:10819000C2B9184BDC6A196B8C420FD01449022407
:1081A0000C61196B4C1C1C63194491F83410C9B252
:1081B0008180196B202905D11A6303E040F22771F1
:1081C00005F0E3F8094803885B060BD540F2266109
:1081D00005F0BAF9074B1A6BDB6A9A4202D1044BDD
:1081E00002225A61BDE819408546704700380140B7
:1081F000000801402C0700206C0F0020680F0020B1
:108200000A4BDA6A196B0132202A08BF00228A421F
:108210000AD0D96A194481F83400DA62044840F27D
:108220002771012205F0B1B8704700BF2C0700206C
:10823000003801400A4B59681A6891420BD05A68BD
:10824000511C59601A44127A02705A68202A04D1CB
:1082500000225A6001E0002070470120704700BFF3
:108260002C070020014B9862704700BF2C070020AC
:10827000044B1A7802F0FF0012B100221A7001209C
:10828000704700BF700F002008B5FCF7D3F8044B0F
:1082900000225A601A60BDE80840FCF7C9B800BF68
:1082A0002C07002010B5441E14F8010F10B1FFF781
:1082B000A7FFF9E710BD00BF684620F007018D4613
:1082C00001B5BDE80140854670470000684620F0D2
:1082D00007018D4601B5124B19781A4679B15B68D2
:1082E000013353600F4B1968013119600E4B196847
:1082F00011B11968013919600023137001E00122DE
:108300001A700A4B1A683AB11A68013A1A601B6867
:1083100013B9074B01221A70BDE80140854670472A
:1083200080070020380A0020680F00206C0F002012
:10833000700F002008B5042004F004FA4FF4FA503E
:1083400004F00CFA012004F00FFA05480321002282
:1083500003F05CFEBDE80840012004F019BA00BF3C
:108360009AC30200014B5868704700BF8007002085
:108370002DE9F04192B0032500244FF0090845484B
:1083800001A9ADF804808DF806508DF8074003F080
:108390005CFC414801A9ADF804508DF806508DF8F9
:1083A000074003F052FC0120014603F0B9FF012110
:1083B0004FF4007003F0C0FF384803F053F8384B17
:1083C00004270793374B3548089380230C934FF4C9
:1083D00080730D934FF480630E9320230F9307A9AE
:1083E0004FF40053109309940A970B94119403F0DF
:1083F000A9F82A48012103F0D0F801264FF46023A0
:10840000294802A9049302948DF80C608DF80D6040
:1084100005948DF8187002F0B3FE23480821324607
:108420002B4602F025FF2048294602222B4602F067
:108430001FFF1D4821462A462B4602F019FF2B46F6
:10844000194841463A4602F013FF224616484FF4B7
:10845000FC6102F0D4FE1448314602F0C7FE124817
:10846000314602F0BAFE104802F0D2FE0E4802F089
:10847000D4FE0028FAD10C4802F0D3FE0A4802F0DC
:10848000D5FE0028FAD10848012102F0D3FE12B02F
:10849000BDE8F08100080140000C014008000240E6
:1084A0004C2401408807002000240140F8B5092829
:1084B00062D8DFE800F005616161086161610C1458
:1084C0003B4B188801E03A4B588880B2F8BD384BD6
:1084D000988840F26B1380B258430013F8BD344BB8
:1084E000D88880B206F0D2FE06F0B4FA0022314BF2
:1084F00006F004FB22A3D3E9002306F0FFFA0446AA
:108500000D4622462B461EA1D1E9000106F042F994
:108510001DA3D3E9002306460F462046294606F050
:1085200017FC02460B463046394606F011FC06F0B1
:10853000A7FD06F08FFA00221F4B06F009FC07F09A
:108540003FFD13A3D3E9002306F0D8FA12A3D3E921
:10855000002306F021F902460B4611A1D1E90001E2
:1085600006F0F6FB10A3D3E9002306F013F906F09A
:1085700087FD07F0A9F8F8BD0020F8BDAFF3008033
:108580006666666666660A409A9999999999014065
:10859000C3F5285C8FA272400000000000FEAA40D4
:1085A0009A999999FD6F2F41C3F5285C8F127140FC
:1085B000880700200000303F00002440AFF3008017
:1085C000014B00221A60704790070020034B9B7AF2
:1085D00013B1034B05225A60704700BF800F002083
:1085E00090070020014B04225A607047900700203A
:1085F000034B1A7A202A04BF00221A72704700BF68
:10860000900700207047212810B508D1104B1B6837
:108610001B7803F07F03212B10D0022010BD2028EF
:10862000FBD10B4B0B4A1B681B78107203F07F03C6
:10863000212B094B18BF00230BB9EEE7074B044A67
:10864000002412682046936154829847204610BD4A
:10865000E00F002090070020AD86000895860008F6
:10866000074B1B681B7803F07F03212B06D100F01A
:10867000DF0002280CBF0020022070470220704754
:10868000E00F002021B9022834BF002002207047EB
:108690000220704720B9034B08221B681A827047DA
:1086A00001487047E00F00204800002020B9034B2C
:1086B00008221B681A82704701487047E00F0020AB
:1086C0004800002008B5032005F0E0FE064B0246F6
:1086D000D8604FF48871054805F08AFCBDE8084071
:1086E000032005F052BD00BF90070020E60F0020D8
:1086F00038B5334B00241B68C0259C725D72DC7258
:10870000204605F0B1FC20464FF4007105F0C9FC8D
:108710002046102105F0DCFC2046402105F038FE03
:108720008021204605F023FE204605F05AFD254B0A
:10873000204693F8341005F078FE204605F025FD1C
:108740000120214605F0ADFC0120294605F00FFE71
:108750000120202105F0BCFC0120214605F0CDFCC4
:1087600002204FF4C06105F09CFC02204FF48071A0
:1087700005F0FDFD0220214605F0BFFC022020216E
:1087800005F0A6FC0320214605F08BFC03204FF4E6
:10879000887105F0FDFD0320402105F046FE032011
:1087A0004FF4405105F0A9FC0320214605F090FC50
:1087B000204605F0BBFA044B01225A6038BD00BFC9
:1087C000E00F00204800002090070020014905F03C
:1087D000A7B800BF80000020014905F0A1B800BF84
:1087E00088000020054B1B68DB78042B04D8044963
:1087F00001EBC30105F094B800207047E00F0020A2
:108800009000002008B5012003F014FDBDE80840E9
:108810004FF40000012103F09BBD024B03225A607C
:10882000704700BF90070020044B9A7A044B0AB1AE
:10883000052200E001225A60704700BF800F00202F
:108840009007002007B514238DF8043000238DF81D
:1088500005308DF8063001A801238DF8073003F0AC
:10886000FFFA03B05DF804FB18B10448102103F0CF
:1088700054BA0248102103F052BA00BF000C014064
:108880007047684620F007018D4679B5154D164BA7
:108890002A681C4692B21A80144A18881188164613
:1088A000014011F4806F05D04FF6FF332B60104B61
:1088B000DB689847238832881340990507D54FF61F
:1088C000FF532B600B4B197C0131C9B219742388FB
:1088D0001A40130401D505F091FABDE879408546A8
:1088E000704700BF445C0040760F00202610002037
:1088F000480000209007002008B50848102103F028
:108900000CFA074B01221A60064A0020064918603B
:1089100010604FF4E0520A801A6008BD000C01405C
:10892000405C0040445C004026100020084B10B51D
:108930001B6800249C72FFF7DFFF064B064A1C6091
:108940004FF406431380054A1360054B5C6010BD6D
:10895000E00F0020445C004026100020405C0040F6
:108960009007002038B5064D01232B60054B0024ED
:108970001C602046FFF778FF03232B60204638BD9C
:10898000405C0040445C0040074B1A6892B242F0E1
:1089900008021A601A6892B242F004021A60034B8D
:1089A00003225A60704700BF405C004090070020DF
:1089B00010B5064C4FF6FB73226813402360FFF797
:1089C00033FF4FF40643236010BD00BF405C0040FE
:1089D00010B51E4C072818BF20702378052B32D8FD
:1089E000DFE803F003060A0E1621FFF7E1FF2AE095
:1089F000FFF7DEFF042327E002236370032323E055
:108A00006378013BDBB263706378F3B9042217E04B
:108A10000F4B1A6892B242F010021A6005232370BD
:108A20000A23637010BD6378013BDBB26370637827
:108A30005BB9074A4FF6EF7311680B4013600622CB
:108A4000024B1A7010BD0623237010BDE40F0020E6
:108A5000405C004007B5FFF7D5FEFFF7F3FE05F0D9
:108A6000B1F90820012103F067FC10230322064816
:108A700001A9ADF804308DF806208DF8073003F019
:108A8000E4F803B05DF804FB000C014007B51423C3
:108A90008DF8043000238DF805308DF8063001A8DC
:108AA00001238DF8073003F0DBF903B05DF804FB18
:108AB000FFF758BF0B4910B5CA6882B14B68052B48
:108AC0000CD10023CC68A34204D2074C1C5DC454D3
:108AD0000133F7E7034B0021D96000E00022104684
:108AE00010BD00BF90070020E60F0020084BDA6899
:108AF000082A1A460AD900230649595CC154013391
:108B0000092BF9D10023D360012070470020704762
:108B100090070020E60F002010B5084C0A4621609F
:108B200092B2C02105F04CFA0120218805F05CFCCE
:108B3000BDE81040012005F019BB00BF90070020E0
:108B4000704710B5FFF70EFC074C2368C01AB0F54C
:108B5000FA7F07D9054BDA6882F40072DA60FFF712
:108B600001FC206010BD00BF28100020000C014057
:108B70007047704770477047054B064AD3F803109B
:108B8000054B09B9928800E0128992B25A60704789
:108B9000C8090020006C00403C0A00207047704764
:108BA0007047704770B50546C5F3074100220120A4
:108BB000FBF7E0FE0A4C0602C5F307210022012064
:108BC0002660FBF7D7FE304306020120E9B20246D9
:108BD0002660FBF7CFFE30430609266070BD00BF5C
:108BE000A407002038B5484C0B2303FB004203FBCD
:108BF000004311790433032984BF032111719A784A
:108C0000032A84BF03229A700B2303FB004203FB59
:108C10000043117A04320F2984BF0F2111715A7A4F
:108C20000433072A84BF07225A710B2303FB004237
:108C300003FB0043917A04320F2984BF0F21917105
:108C40005A7B0C330F2A84BF0F225A700B2202FB6F
:108C5000004302FB0042997B0C330F2984BF0F2194
:108C6000997013795279DB0343F4002121611AB121
:108C7000254943F404230B610B2101FB0041C97911
:108C8000214B19B1196941F4005119610B2372B9D3
:108C900003FB0043197A9A79C90141EAC2210433DE
:108CA00022695B790A4342EA031222611AE003FB5C
:108CB00000431B7B144A1BB1136943F480531361B7
:108CC0000B2202FB0042917B557B22690E4B42EA4C
:108CD000C51201F0070542EA0512090748BF42F430
:108CE00000621A610B2202FB0040C27A064B04307C
:108CF0001AB91A6981790A431A612069FFF752FF8C
:108D00002369636138BD00BFA407002010B5114C72
:108D10000023C000236123185B7F13B14FF400735D
:108D200023612218927F0B4B1AB11A6942F48072A8
:108D30001A612318DA7F20440F2A84BF0F22DA77C2
:108D4000C07F236918432061FFF72CFF236923624A
:108D500010BD00BFA407002010B5224C4FF46023C3
:108D6000C0002361231893F82B3013B14FF4702304
:108D70002361231893F8252093F82410120342EA64
:108D8000813293F826302169012B42EA01022261E7
:108D900003D1144B42F480621A61221892F8271012
:108DA000236992F8282043EA0123012A236103D191
:108DB0000C4A43F080031361221892F82920094BD2
:108DC000012A03D11A6942F040021A612044236942
:108DD00090F82A0043EA00102061FFF7E3FE2369C0
:108DE000E36210BDA407002038B52A4C43001A18CE
:108DF000224492F9311030323F29C4BF3F215170D3
:108E00001A18224492F9311030323F31BCBFC121CF
:108E100051701A18224492F8321030321F2984BF40
:108E20001F2191704FF4402222611A18224492F8B7
:108E30003020012A03D1174A4FF45021116104EB6D
:108E4000C00191F82B10134A51B91918114491F827
:108E50003150116905F07F0541EA052111610CE0EF
:108E60001D18154495F8315001F0030105F07C05FB
:108E70002943156945EA012515610344234493F804
:108E80003200236918432061FFF78CFE2369636376
:108E900038BD00BFA407002010B58300244C1A1869
:108EA000224492F83810012984BF012182F8381039
:108EB0001A18224492F839103832032984BF03214A
:108EC00051701A18224492F83A1038320F2984BF90
:108ED0000F2191701A18224492F83B10383203295E
:108EE00084BF0321D1701A18224492F83C10034425
:108EF0000F2902F1380284BF0F211171234493F826
:108F00003C0003F1380293F8383040F4202040EA66
:108F1000C330537840EA4330937840EA0320D37853
:108F200040EA43102061FFF73DFE2369236410BD32
:108F3000A4070020224B012210B50521002483F84C
:108F400030200220032283F8264083F8274083F84C
:108F5000284083F8294083F82A0083F82B4083F8BF
:108F6000384083F8394083F83A4083F83B4083F82F
:108F70003C405C779C77DC7718715C71DC719C718C
:108F80001872DC721C735C7383F8311083F8321032
:108F900083F8242083F825205A7299729A73204608
:108FA000FFF77AFF2046FFF71FFF2046FFF7D4FEAA
:108FB0002046FFF7ABFE2046BDE81040FFF712BE8B
:108FC000A4070020054B042903EBC00318BF0022AF
:108FD000D97718BF5A77FFF799BE00BFA4070020C2
:108FE000044B03EBC003597709B10422DA77FFF78A
:108FF0008DBE00BFA4070020024B03EBC00399778E
:10900000FFF784BEA4070020024B03EBC000C07F23
:10901000704700BFA4070020024B03EBC000407F55
:10902000704700BFA4070020024B03EBC000807F05
:10903000704700BFA4070020034B0B2202FB003344
:109040001971FFF7CFBD00BFA4070020034B0B220F
:1090500002FB00335971FFF7C5BD00BFA407002014
:10906000034B0B2202FB0033D971FFF7BBBD00BFDE
:10907000A4070020034B0B2202FB00339971FFF77A
:10908000B1BD00BFA4070020034B0B2202FB00333D
:109090001972FFF7A7BD00BFA4070020034B0B22E6
:1090A00002FB00335972FFF79DBD00BFA4070020EB
:1090B000034B0B2202FB00339972FFF793BD00BFF5
:1090C000A4070020034B0B2202FB00331973FFF7A8
:1090D00089BD00BFA4070020034B0B2202FB003315
:1090E0005973FFF77FBD00BFA4070020034B0B227D
:1090F00002FB00339973FFF775BD00BFA407002082
:10910000024B0B2202FB003000797047A4070020BD
:10911000024B0B2202FB003040797047A40700206D
:10912000024B0B2202FB0030C0797047A4070020DD
:10913000024B0B2202FB003080797047A40700200D
:10914000024B0B2202FB0030007A7047A40700207C
:10915000024B0B2202FB0030407A7047A40700202C
:10916000024B0B2202FB0030807A7047A4070020DC
:10917000024B0B2202FB0030007B7047A40700204B
:10918000024B0B2202FB0030407B7047A4070020FB
:10919000024B0B2202FB0030807B7047A4070020AB
:1091A000034A00EB8003134483F83810FFF774BEC2
:1091B000A4070020034B00EB800213445970FFF713
:1091C0006BBE00BFDC070020034B00EB80021344A2
:1091D0009970FFF761BE00BFDC070020034B00EB76
:1091E00080021344D970FFF757BE00BFDC07002090
:1091F000034B00EB800213441971FFF74DBE00BF13
:10920000DC070020034B00EB8000184490F8380086
:10921000704700BFA4070020024B00EB80001844F9
:1092200040787047DC070020024B00EB80001844B8
:1092300080787047DC070020024B00EB8000184468
:10924000C0787047DC070020024B00EB8000184418
:1092500000797047DC070020034A00EB4003134409
:1092600083F83010FFF7C0BDA4070020034B00EBCC
:10927000400213445970FFF7B7BD00BFD407002068
:10928000034B00EB400213449970FFF7ADBD00BFE4
:10929000D4070020034B00EB4000184490F8300046
:1092A000704700BFA4070020034B00EB40001844A8
:1092B00090F90100704700BFD4070020024B00EB7B
:1092C0004000184480787047D4070020034B03EB1C
:1092D000C00383F82410FFF73FBD00BFA4070020A0
:1092E000034B03EBC00383F82510FFF735BD00BF28
:1092F000A4070020034B03EBC00383F82610FFF7FD
:109300002BBD00BFA4070020034B03EBC00383F871
:109310002710FFF721BD00BFA4070020034B03EB7C
:10932000C00383F82810FFF717BD00BFA407002073
:10933000034B03EBC00383F82910FFF70DBD00BFFB
:10934000A4070020034B03EBC00383F82A10FFF7A8
:1093500003BD00BFA407002010B5064B044603EB75
:10936000C00383F82B10FFF7F7FC2046BDE8104040
:10937000FFF73ABDA4070020024B03EBC00090F8B2
:1093800024007047A4070020024B03EBC00090F8B4
:1093900025007047A4070020024B03EBC00090F8A3
:1093A00026007047A4070020024B03EBC00090F892
:1093B00027007047A4070020024B03EBC00090F881
:1093C00028007047A4070020024B03EBC00090F870
:1093D00029007047A4070020024B03EBC00090F85F
:1093E0002A007047A4070020024B03EBC00090F84E
:1093F0002B007047A40700202DE9F0472E4D1E4694
:109400002B1893F8443004468A469146DDF82080B4
:10941000099F042B1AD8DFE803F003080D12170088
:10942000FFF7E0FB2B19012212E0FFF795FC2B1947
:1094300002220DE0FFF730FD2B19032208E0FFF7B1
:10944000D3FC2B19042203E0FFF760FC2B19002248
:1094500005EBC40483F8442094F82A20164B012A13
:1094600013D002D3022A15D021E0BAF1000F03D0A5
:109470001B689B0C8AF80030B9F1000F17D02B68DD
:10948000C3F38923A9F8003011E086B11B689B0A59
:1094900033600CE01EB11B68DB0B5B013360B8F17D
:1094A000000F04D02B68C3F3842388F800300FB179
:1094B0002B683B70BDE8F087A407002030B9044B4F
:1094C000DA7A1AB90122DA72FFF78CBB704700BF53
:1094D000A407002028B9034BD97A11B1D872FFF73D
:1094E00081BB7047A40700202DE9F041114AC70055
:1094F000D31993F82A600546032E904604D0032220
:1095000083F82A20FFF728FC2846FFF725FCD8F827
:109510000040230344BF6FEA04346FEA1434032E7F
:1095200005D0474487F82A602846FFF715FC2046F7
:10953000BDE8F081A407002070B5084C9DF81060CC
:109540009DF8145004EBC00421766276A376E6768B
:109550002577BDE87040FFF7D9BB00BFA407002006
:1095600006281AD8DFE800F004070A0D10131600C9
:109570000A4B1B6810E0094B1B6A0DE0074B5B6947
:109580000AE0064B1B6C07E0044B5B6B04E0034BEB
:10959000DB6A01E0014BDB7A0B607047A407002017
:1095A000014B1878704700BFEC070020034B0020E8
:1095B0001870034B997AFAF731BF00BF2F0F0020C4
:1095C000C80E00202DE9F04F8D4C87B0637823B989
:1095D0006FF00043636001236370257A894F4DB9B2
:1095E000E8B2FAF7C8FE78550135082DF8D1844B5A
:1095F00001221A7227250026F0B2FAF7BCFEBB5DE5
:1096000083421AD07F4B321DF0547F4B53F82230E7
:10961000022B05D0032B0AD0012B0ED168B106E036
:1096200058B97A4A515D012907D1535505E0774B66
:109630005A5D012A04BF02225A550136082E05F14F
:109640000105D9D1724EF36993B1724D2F787FB96C
:10965000FEF788FE704B1B68C01AF3690028B8BF7C
:109660004042984204D9384601F078F901232B7022
:10967000336AA3B1694D2E788EB9FEF773FE684B3D
:10968000634A1B68126AC01A80EAE073A3EBE073B6
:10969000934204D9304601F061F901232B70607CBC
:1096A000604D574E05EB40131F7B002F00F0FB80F1
:1096B0005D4B5E4F03440093C31901935C4B002143
:1096C00003EB80030A46FFF797FE707C4301EA181C
:1096D000127B013A042A00F2D480DFE802F0033A58
:1096E000AF3AAF00534A544E926812F0200F04EB89
:1096F0000002927C10D0022A03D1325C002A00F0D2
:10970000C0801D44697AFAF789FE607CFFF7E2FEAB
:10971000637C0221E21818E0012A03D1325C002A9E
:1097200000F0AF802B44997AFAF778FE607C05EB65
:109730004015AB7A13B9FFF7C1FE03E0335C0BB100
:10974000FFF7C8FE637C0121E21891740022F254F5
:1097500097E03A56384E002A19DB2218927C022AEA
:1097600001D1325C62B12B44597AFAF757FE607C22
:10977000FFF7B0FE637C0221E21891740022F254DC
:10978000667CFEF7EFFD04EB8606706032E0204455
:10979000837C1B4F012B03D1637CF35C93B929E0DD
:1097A000FEF7E0FD7B7C0A2107EB830705EB431303
:1097B0009B8B7A684B43801A80EAE072A2EBE072DE
:1097C0009A42E9DD607C05EB4013997AFAF726FEB0
:1097D000607C05EB40139B7A13B9FFF76FFE03E043
:1097E000335C0BB1FFF776FE637C0121E2189174C4
:1097F0000022F254637C05EB43152B7B042B36E0EF
:10980000EC070020F5070020F00E0020360F0020A6
:10981000080000202D0F0020280F0020510E0020EE
:10982000200F0020C80E00205A0E0020C10E00207C
:10983000700E0020000C01402C0F00202218927C9A
:109840008C4E022A01D1325C62B12B44597AFAF76C
:10985000E5FD607CFFF73EFE637C0221E218917417
:109860000022F254637C05EB43152B7B052B08D1BA
:10987000814B9A6812F0200F4FF4806214BF5A6136
:109880001A61FEF76FFD6369C01A80EAE073A3EB0B
:10989000E0730A2B40F3D582FAF73AFEFEF762FD39
:1098A000764B5861CDE2FAF733FEFAF7B1FF88B98B
:1098B000367886B9724F00F091FD304601F04EF8CF
:1098C0003B7823B13046A97AFAF7A8FD3E70012310
:1098D000237000E03770FEF745FD6369674FC01ADB
:1098E00080EAE073A3EBE0730A2B40F3AA82387896
:1098F000002840F0A082797C490141F00A0101F082
:10990000EA0100F0F8FE0646787C002840F0F3817A
:1099100001F06CF9787C0C2242435A49584F8B185D
:10992000D3F804808A581B7ADFF85C91002B18BFAB
:1099300090463B5C032B00F2B980DFE803F0025C49
:10994000153B002E00F0B28005EB4013D97F21B10A
:10995000FAF764FD637C032204E0597AFAF75EFDAE
:10996000637C0222FA54A1E04EB9400140F00801A4
:1099700001F0E801304600F0BEFE002845D086EA3E
:10998000E673A3EBE673B8F1000FB8BFC8F10008A7
:109990004345607C01D0002E78D159F830209342A5
:1099A0007ED2394B03EBC0031979FAF737FD334BFD
:1099B0005B7C17E086EAE673A3EBE673B8F1000F71
:1099C000B8BFC8F10008434501D0002E68D159F84E
:1099D0003020934208D22C4B03EBC0031979FAF7DD
:1099E0001DFD637C01225AE005EB4013597AFAF71A
:1099F00015FD637C3CE01EBB400140F0080101F016
:109A0000E801304600F077FED0B9FEF7ABFC637C8E
:109A10004FF00A0E04EB83025268801A05EB4312E2
:109A2000918B0028B8BF40420EFB01F188423DDD1A
:109A30001846917AFAF7F2FC104B5B7CFE5435E045
:109A400086EAE673A3EBE673B8F1000FB8BFC8F17E
:109A500000084345607C00D0C6B959F830209342D5
:109A60001ED305EB4013597AFAF7D8FC034B5B7C05
:109A7000022214E02C0F0020000C0140EC07002013
:109A80002F0F0020780E00205C0E002005EB401305
:109A9000D97F29B1FAF7C2FC864B03225B7CFA54CA
:109AA000677CFEF75FFC04EB87077860607C824B85
:109AB000002103440093814B0A4603440193804BE9
:109AC000DFF8F08103EB8003FFF796FC607C7D4FAD
:109AD00005EB40139B694BB3FAF796FC30B398F84B
:109AE000110086EAE672A2EBE67207EB40139B696F
:109AF0009A421BD900F032FF98F81130724A0121C6
:109B0000D15407EB43139B7F43B1BA7F9A4205D1EF
:109B1000002000F023FF002000F060FC637C6B4A13
:109B20000F33D15C012904BF0221D154627CDFF8DC
:109B3000848151016B185B69DFF888A1002B6AD022
:109B4000634B9F5C9B46002F65D1002E64D041F093
:109B5000020101F0E201384600F0B4FF024698F835
:109B600011000392FAF79AFD98F81110039A0AEB84
:109B700041135B69101A80EAE072A2EBE07283EA9B
:109B8000E37EAEEBE37E724554DD002B10DD08462C
:109B900000F0E4FE98F811300AEB43139B7F5BB3AF
:109BA0009AF81E209A4227D1384600F0D7FE20E0CE
:109BB0003846022200F0B7FD98F8111038464901E6
:109BC00041F0080101F0E80100F062FD98F8113061
:109BD0000AEB43139B7F7BB19AF81E209A420BD16C
:109BE00038463946022200F09EFD3846082100F032
:109BF0004FFD384600F0F2FB607C344A00F115035B
:109C0000D15C012904BF0221D15401230BF800309B
:109C100000F0E4FB0EE06EB941F00801002001F015
:109C2000E80100F068FD28B9637C05EB4312D28996
:109C300062B10EE0677C274BDB5D002BF4D1FEF7B1
:109C400091FB1C4B03EB8707B8611EE0214AD35CF4
:109C5000DBB1FEF787FB637C04EB8302926905EBC3
:109C60004315801AE98980EAE072A2EBE0720A20CB
:109C700041438A4209DD184DEA5C32B91846FFF7C4
:109C80001DFC0C4B01225B7CEA54607C002EB8BFAB
:109C9000764259F83030074F9E42104D20D2FFF7E0
:109CA000D3FA7B7C05EBC3056A79824223D118463F
:109CB00000211EE0EC0700205A0E0020C10E0020FB
:109CC000700E0020C80E0020C00E0020360F0020AD
:109CD000650E0020340F0020350F00205C0E0020A0
:109CE000FFF7B2FA7B7C05EBC3056979884202D0A5
:109CF0001846FFF77DFA002000F0E1FC227FC7073D
:109D000002F0F802504B48BF42F0010246071A77B2
:109D100003D5237F43F002032377C50603D5237FB2
:109D200043F004032377494B1A78D10715D5227FD6
:109D3000D20712D5464A1178CF070ED441F001015F
:109D40001170444A117841F001011170424A012119
:109D50001170424A127802B91A70237FDE0709D5C2
:109D6000394A527FD50705D43D4AD178012904BF2D
:109D70000221D170990708D5627F920705D4384A2D
:109D80001179012904BF022111715F0708D5627F93
:109D9000560705D4324A5179012904BF0221517175
:109DA00005066377617C43D5490141F01601002027
:109DB00001F0F60105AA00F087FC9DF81630580660
:109DC00009D5214A2649527C52001B32885C012861
:109DD00004BF02208854190609D5617C204A0E313F
:109DE00012F81100012804BF022002F81100DA065F
:109DF00008D5627C1A4952001B32885C012804BFD6
:109E0000022088549B0609D5627C154B0E3213F84C
:109E10001210012904BF022103F81210617C0020F6
:109E2000490141F0160101F0F60105AA00F080FB9E
:109E3000607C00F017F8044B00225A74FEF792FA87
:109E4000606107B0BDE8F08FEC0700206C0E0020C9
:109E5000590E0020660E0020650F0020580E0020CD
:109E6000360F00202DE9F04F4FEA401887B05FFA17
:109E700088F5044645F07C0105AA002000F024FC8A
:109E8000B54B4FEA440A03EB0806307A022110F082
:109E9000400F9C4672689DF8163001FA0AF10DD009
:109EA0004FF0010B0BFA0AFB194003EA0B0B5CF8AD
:109EB0000830C2F100095B42039309E001EA030B99
:109EC000012101FA0AF119405CF808309146039328
:109ED000A24B10F0800F9B6800F03F0718BF83F083
:109EE0002003781EC3F34013072800F26782DFE8DF
:109EF00010F008000800080008001C011C011C01EB
:109F00001C01974E335D0F2B00F25882DFE813F0EF
:109F10005602100054013C007C01480051005D00D5
:109F20007000A100D900DE005602F80001014002D5
:109F300045F0140105AA002000F0C6FB45F0060517
:109F40009DF8153006EB840629460020736000F06A
:109F5000D2FB2146B0600222002000F0E4FB00208A
:109F6000294640F2FF7200F008FB00202146032240
:109F700000F0FBFB023F012FDFF8E48194BF0223D6
:109F8000042308F8043019E2002900F017820020A9
:109F900045F0020100F096FD724B43F824002AE1DF
:109FA000BBF1000F00F00A82204600F0D7FC062328
:109FB00003E221460020032200F0D7FB002045F0F9
:109FC00008014A4600F0D9FA47E1BBF1000F40F022
:109FD000F58145F00805584629465A4600F0CDFA65
:109FE00058462946C9F1000200F0C7FA0823E4E107
:109FF000BBF1000F00F0E28145F00201002000F00B
:10A0000061FD07460020024645F0080100F0B5FA60
:10A01000544B002053F824202146D21B43F824201F
:10A02000032200F0A2FB002045F0060189EAE97254
:10A03000A2EBE97200F0A1FA002008F0E0013A4634
:10A0400000F0ADFA00202146024600F06CFB092327
:10A05000B3E1002000F033FB40FA0AF0C10740F101
:10A06000AD8145F0020A5146002000F02BFD3E4B29
:10A0700045F0080543F8240000200246294600F078
:10A080007CFA00202146022200F04DFB002002460F
:10A09000514600F084FA0020024608F0E00100F08A
:10A0A0007EFA033F20460021FAF70CFB012F00F255
:10A0B0007A8100202146022200F035FB002029464B
:10A0C000F7E0BBF1000F40F0048177E1BBF1000F36
:10A0D00040F0748145F00201584600F0F3FC45F071
:10A0E000080107465A46584600F047FA02225846E9
:10A0F00008F0E00197FBF2F200F051FA584614E143
:10A10000002000F0DCFA40FA0AF0C20740F1568164
:10A1100049E106EB8407002045F00601BA6800F02B
:10A120002CFA002021463A7944E10D4E305D0F288B
:10A1300000F24481DFE810F042011A003E005900AD
:10A14000660082004201930042014201C300CF0039
:10A15000A900FF0039012C01C80E0020000C0140AD
:10A160000C080020540E0020EC0E002045F01401D5
:10A1700005AA002000F0A8FA9DF8152006EB84033C
:10A180005A6000202146022200F0CDFA002045F05E
:10A19000060140F2FF7200F0F0F900202146032290
:10A1A00000F0E3FA062F51D0082F4FD0854B042240
:10A1B0001A5503E1062F09D106EB84035A680020E3
:10A1C00002F00402214642F0010204E0082F04D10B
:10A1D00000202146032200F0C8FA002045F00801C3
:10A1E000039A00F0CAF90323E7E07A1F012A04D892
:10A1F00019B1062F2CD10423DFE0002B00F0DE8004
:10A200000C23DAE0052F09D106EB84035A680020FD
:10A2100002F00402214642F0020204E0072F04D1BA
:10A2200000202146032200F0A0FA039B00205A429E
:10A2300045F0080100F0A1F90523BEE07A1F012ACC
:10A2400008D8BBF1000F05D0052F01D10223B4E0DF
:10A250000F23B2E0002B00F0B1800723ADE0002B0C
:10A2600040F0AC80073F012F0AD906EB8402526808
:10A27000184602F00402214642F0010200F075FA8D
:10A28000002045F008014A4615E0002B40F096807A
:10A29000073F012F0AD906EB84025268184602F0E4
:10A2A0000402214642F0020200F05FFA002045F06D
:10A2B0000801C9F1000200F060F90A237DE0002BDB
:10A2C0007CD0002045F0020100F0FCFB06EB84038B
:10A2D000D8600B2371E0002B70D1184645F00201C5
:10A2E0000193CDF808C000F0EDFBDDF808C0019B3C
:10A2F0000CEB08025373074645F00601184689EA3D
:10A30000E972A2EBE972019300F049F906EB8402CD
:10A31000D268019B17440222184608F0E00197FB1F
:10A32000F2F200F03CF9019B18462146024600F08B
:10A33000FAF90D2341E0002000F0C1F940FA0AF0DB
:10A34000C3073BD50E23335545F0020631460020A6
:10A3500000F0B8FB1C4B45F0080143F82400002036
:10A36000024600F00AF921460020022200F0DBF943
:10A3700000203146024600F012F9002008F0E0010A
:10A38000024600F00CF920460021FAF79BF915E08F
:10A3900000202146022200F0C6F9002045F0080105
:10A3A000024600F0EAF80E2307E006EB84031A7970
:10A3B0000020214600F0D9F90023335507B0BDE84D
:10A3C000F08F00BF0C080020EC0E0020024B1A5C3E
:10A3D0000AB901221A5470470C080020024B1A5C7B
:10A3E0000AB10F221A5470470C080020014B185C68
:10A3F000704700BF0C0800202DE9F0411446127888
:10A400000746C2F341150E466DBB444901EB4511A9
:10A4100001F10803187930BBD00724D45F2A22D871
:10A420003F48405DF8B912F0970F1CD1DFF8F88073
:10A4300018F8050060B9C97F19B1F9F7EFFF0323D8
:10A4400004E008465978F9F7E9FF022308F80530D7
:10A45000DFF8D88018F805302BB10020FFF73AF864
:10A46000002308F80530217800220220FAF782FA4A
:10A470003070617800220220FAF77CFA7070A178BF
:10A4800000220220FAF776FAB07001220220E17869
:10A49000FAF770FAF0702378DA073DD45F2B3BD8D7
:10A4A00003F01E02082A12D0142A2BD0062A33D118
:10A4B000242257435B090C2202FB0373A178E27844
:10A4C000184F42EA01223B445A60BDE8F081242142
:10A4D00079435B090C2000FB0313A678E578114A49
:10A4E00045EA0625D550A3781B0715D527787F099F
:10A4F00000FB0717D3596FEA03536FEA1353D35185
:10A50000BDE8F08124214F435B090C2101FB03735B
:10A51000044FE2783B441A72BDE8F081C80E002077
:10A52000340F0020780E00202F0F0020350F002060
:10A5300007B513788DF800108DF80130537801A914
:10A540008DF8023093786A468DF80330FFF754FF98
:10A5500003B05DF804FB07B58DF802309DF81030AC
:10A560008DF800108DF8012001A96A468DF803309E
:10A57000FFF742FF03B05DF804FB07B500238DF839
:10A5800000108DF801308DF80320131201A96A46DE
:10A590008DF80230FFF730FF03B05DF804FB5F2950
:10A5A0002DE9F34105460E46144658D811F01E0712
:10A5B000C1F3411202D0022F1DD050E000EB400346
:10A5C0001A4430491201881843688C50C3EB040EBA
:10A5D000BEF1000FB8BFCEF1000EBEF5000F08DBD4
:10A5E0009C42CCBF284C294C0A441C4401231373C1
:10A5F00035E0077333E000EB4007224B17443F017F
:10A60000D91924F07F4EC1F808E04C6001F1080030
:10A61000D9599846C4EB010EBEF1000FB8BFCEF178
:10A62000000EBEF5000F18DBA142CCBF164B174B36
:10A63000520123448DF800201A148DF801201A12BB
:10A640008DF80220284601A96A468DF80330474458
:10A65000FFF7D2FE01233B7301E0002303712314B3
:10A660008DF801302846231201A96A468DF8006052
:10A670008DF802308DF80340FFF7BEFE02B0BDE852
:10A68000F08100BF2C100020FFFF7F00010080FF41
:10A6900007B511F01C0202D1FFF781FF0CE0002387
:10A6A0008DF800106A4601A98DF801308DF802304E
:10A6B0008DF80330FFF7A0FE03B05DF804FB012125
:10A6C00002200A46FAF756B913B541F001011446C3
:10A6D0008DF8041001AA6946FFF78EFE9DF801303F
:10A6E0009DF8000023709DF8023063709DF80330E0
:10A6F000A37002B010BD07B541F001018DF8041040
:10A7000001AA6946FFF778FE9DF803309DF8020024
:10A7100043EA0020030544BF6FEA00506FEA10507F
:10A7200003B05DF804FB73B54901CCB244F01503E6
:10A73000164601A96A4605468DF80030FFF75CFE13
:10A740009DF8053044F014048DF801309DF8063072
:10A75000284601A96A468DF800408DF802308DF830
:10A760000360FFF749FE02B070BD73B54901CCB27A
:10A7700044F01503164601A96A4605468DF80030D7
:10A78000FFF73AFE9DF8053044F014048DF80130CF
:10A790009DF80730284601A96A468DF800408DF8DB
:10A7A00002608DF80330FFF727FE02B070BD2DE97F
:10A7B000F3474001C7B2C1F30A06002047F0180171
:10A7C00001AAFFF781FF9DF8058030464FEA18196E
:10A7D00008F00F08C8450FDB04F01AF9C9EB0808A8
:10A7E0000446012000FA08F00D4604F021F9002289
:10A7F000354B04F083F910E004F00AF9C8EB0908BE
:10A800000446012000FA08F00D4604F011F9024652
:10A810000B4600202C4904F09BFA02460B462046CA
:10A82000294604F095FA04F02BFC04F013F924A354
:10A83000D3E9002304F062F904F022FC04F00AF9E1
:10A840000022224B04F05AF94FF0FF3904460D461E
:10A85000CA464FF00008012000FA08F004F0E8F8BA
:10A8600002460B462046294604F048F904F0E0FB76
:10A87000A0F18002802A38BFC14608F1010828BF34
:10A880005046B8F10E0F01D08246E4E700248DF85F
:10A89000050047F01201204601AA8DF804408DF80A
:10A8A0000690FFF745FE204647F00C013246FFF7C1
:10A8B00064FE204602B0BDE8F08700BFAFF3008021
:10A8C00004560E2DB29DEF3F000060400000204076
:10A8D00073B54C0804EB4404B42304F5807403FB03
:10A8E0000044054620460E46FDF7C6FA8DF80400E2
:10A8F000601CFDF7C1FA8DF80500A01CFDF7BCFA3D
:10A9000046EA45118DF80600C9B2002001AAFFF7FA
:10A910000FFE02B070BD37B50C46640841EA401125
:10A9200001AA0546C9B2002004EB4404FFF7CCFE9F
:10A9300004F58074B42303FB05449DF804102046FD
:10A94000FDF7C1F9601C9DF80510FDF7BCF9A01CCE
:10A950009DF80610FDF7B7F903B030BD10B5C4B2CD
:10A9600021466401E4B200200222FFF7DCFE44F03D
:10A9700008010020FFF78CFE44F00A010020BDE82A
:10A980001040FFF785BE37B5400140F01604E4B231
:10A990000D4601AA21460020FFF796FE9DF80530DE
:10A9A00015F0010F14BF43F0400323F040038DF86E
:10A9B00005309DF8053015F0020F14BF43F0100369
:10A9C00023F010030020214601AA8DF805308DF8F0
:10A9D0000600FFF7ADFD03B030BD37B5400140F0D4
:10A9E0001604E4B20D4601AA21460020FFF76CFED2
:10A9F0009DF8053015F0010F14BF63F07F0303F0DD
:10AA00007F038DF805309DF8053015F0020F14BF57
:10AA100043F0200323F020030020214601AA8DF8F3
:10AA200005308DF80600FFF783FD03B030BD07B594
:10AA3000400140F0160101F0F60101AA0020FFF7E5
:10AA400043FE9DF80530C3F38010DB0648BF40F09D
:10AA5000020003B05DF804FB07B5400140F01601A9
:10AA600001F0F60101AA0020FFF72EFE9DF8053047
:10AA7000D8099B0648BF40F0020003B05DF804FB14
:10AA800070B50F4C000123189A68914209DD8A1AAB
:10AA9000C2F18075AA425E6801DC324409E0751B90
:10AAA0000AE00ADA521AC2F18075AA425E6802DC34
:10AAB000B21A5A6001E035445D602044816070BD87
:10AAC0002C10002037B541F001030C4601AA69465D
:10AAD0008DF804300546FFF78FFC9DF802309DF895
:10AAE00001201B0243EA02439DF8032043EA0201CE
:10AAF0000B0248BF41F07F415F2C19D8C4F34112CB
:10AB000014F01E040ED0022C12D105EB450515449D
:10AB1000E8B221F07F41FFF7B3FF074B03EB0515C8
:10AB2000696805E005EB45052A44034B1201995875
:10AB3000084603B030BD00BF2C10002038B50C46CD
:10AB400068210546FFF7BEFF14B140F0010201E0A5
:10AB500020F0010228466821BDE83840FFF71FBDFC
:10AB600038B50C4668210546FFF7ACFF14B140F03C
:10AB7000100201E020F0100228466821BDE83840AC
:10AB8000FFF70DBD13B5184B00245A7E93F82830FB
:10AB900012F0010F14BF21222022DB0748BF42F030
:10ABA000100200206821FFF7FAFC009420467E2165
:10ABB00020222346FFF7CFFCE1B200200134FFF74B
:10ABC00087FE1D2CF8D10C210020FFF77BFF0146EA
:10ABD0000020FFF7ECFD0020162143F2FF1202B027
:10ABE000BDE81040FFF7C9BC08000020F0B54501E2
:10ABF00085B0044645F0030303AA002002A98DF89E
:10AC00000C30FFF7F9FB9DF80A109DF80930090296
:10AC100041EA03419DF80B3020461943FFF730FF0E
:10AC200015482301C21802F108010E790EB3134E24
:10AC30000C2707FB0464247ADCB9C6585268B71A9B
:10AC4000002FB8BF7F42B7F5000F05DB9642CCBF9F
:10AC50000B4B0C4B134401E0C3580C71DAB2009259
:10AC60000020C3F3074205F0E001C3F30723FFF719
:10AC700072FC05B0F0BD00BF2C100020780E002043
:10AC8000FFFF7F00010080FF074B10B518681C46CE
:10AC900001460A780B4601311AB12C2AF9D100225B
:10ACA0001A700133236010BD1C08002070B5124BD0
:10ACB00006461B78E3B1FDF7BDFA104C054618B106
:10ACC00000232371012070BDA368E268934207D27C
:10ACD0005A1C23441B7C012033702071A26070BD7C
:10ACE00004F11000FDF7E6FEA560E060284670BDA7
:10ACF000BDE87040FDF79EBA500E00201C080020F1
:10AD000010B50E4B1B7813B10D4C23791BB9BDE860
:10AD10001040FDF775BA226D0D2802F1010322449F
:10AD2000236582F8540002D03F2B00D829B9194678
:10AD30000448FDF7F1FE0023236510BD500E0020EE
:10AD40001C0800207008002070B50121044686B060
:10AD50002020FFF7D5FF002C04DA2D200121FFF77A
:10AD6000CFFF644200230A2194FBF1F201FB124160
:10AD700001AE30311D46995514460133002AF2D1F7
:10AD8000705D0121FFF7BCFF15F1FF35F8D206B069
:10AD900070BD2DE9F34105460DF10700FFF786FF71
:10ADA000974C002800F0C88094F894309DF8070074
:10ADB000944E03BB7378403398420DD1D4F8983049
:10ADC000002B40F0B9803179012331F0010184F882
:10ADD000943040F0B180ADE00D2801D01B2801D1A6
:10ADE000002305E0D4F898307E2B00F2A5800133D3
:10ADF000C4F89830A0E0317931F0010101D1FFF7BA
:10AE00007FFF9DF807301F2B0CD9D4F898207C4980
:10AE10007E2A00F28280501C0A44C1F8980082F811
:10AE20009C307AE0082B08D1D4F89830002B74D0ED
:10AE3000734A013BC2F898306FE00D2B6DD1D4F806
:10AE40009830002B69D03379112B16D16D4B01212D
:10AE5000587800274030C0B2FFF752FFD4F898303E
:10AE60009F4206D2684B0121D85DFFF749FF0137A9
:10AE7000F4E70D200121FFF743FF0023D4F8988069
:10AE80002768C4F81C311A461946424537D00129B3
:10AE900011D002D3022925D02FE0DFF864C10CF1D4
:10AEA0009C00105C202828D00CEB030181F82001C5
:10AEB0000133012121E0524800F19C0C12F80CC032
:10AEC000BCF1200F0AD1012B04D91844002180F8CD
:10AED000201101334D4F02211F440EE0184480F829
:10AEE00020C109E0DFF818C10CF19C00105C20289B
:10AEF00003D09C448CF8200101330132C5E70022C5
:10AF0000C4F81C31234483F820210123276084F8EE
:10AF10009F3184F89420C4F898209DF807301B2BAB
:10AF20000AD133790021012BC4F8981084F89410C9
:10AF300002D10D20FFF7E4FE94F89F0100260028BF
:10AF40005AD02F4B83F89F61F7B2DFF8DC80C7EB54
:10AF5000C70708EB07042D48214604F079FF28B9FC
:10AF6000A6796379F1072B7036D506E018F807301B
:10AF70000136002BE8D12B703DE0FFF785FE2B78E2
:10AF80000446042B14D1224904F062FF08B90023BF
:10AF90000CE020461F4904F05BFF08B9012305E0DF
:10AFA0001D49204604F054FF90B902236B7013E052
:10AFB0000D2B0ED1194904F04BFF0028E7D0204695
:10AFC000174904F045FF0028E8D020461549E9E775
:10AFD000204604F039FF6870B20704D5FFF754FE2D
:10AFE00004F032FFA870730705D5FFF74DFE04F09B
:10AFF0002BFFC5F80300012002B0BDE8F08100BFBF
:10B000001C08002008000020B80800203C0900208F
:10B0100002070108060701080A07010810070108CE
:10B02000160701081B0701080506010838B50D4D74
:10B030000446A87801214030C0B2FFF761FE68786D
:10B0400001214030C0B2FFF75BFE2078FFF77CFEA5
:10B050006068FFF779FEBDE838400D200121FFF759
:10B060004FBE00BF080000207047FEE7FEE7FEE786
:10B07000FEE77047704770477047704770477047EA
:10B080007047704770477047704770477047704708
:10B09000704770477047704770477047704708B5F2
:10B0A000014B1B68984708BD680E002008B5024B8D
:10B0B0001B68984708BD00BF300F002008B5024B41
:10B0C0001B68984708BD00BFC40E002008B5024B9E
:10B0D0001B68984708BD00BFE80E00207047704706
:10B0E00070477047704770477047704770477047A8
:10B0F0007047704770477047704770477047704798
:10B100007047704770477047704770477047704787
:10B110007047704770477047704770477047704777
:10B1200070477047704700BF08B5144B98420FD066
:10B1300003F5A053984213D0A3F5C05398421BD1F6
:10B140004FF40070012101F00FF94FF400700EE090
:10B150004FF48060012101F007F94FF4806006E0B0
:10B160004FF40040012101F0FFF84FF400400021AE
:10B17000BDE8084001F0F8B808BD00BF0028014054
:10B1800043680A6823F4702323F4807313430A7915
:10B1900010B543EA022343608A68CB6884681A4387
:10B1A000084B234013434A7943EA420383600B7CF4
:10B1B000C26A013B22F47002DBB242EA0353C3626B
:10B1C00010BD00BFFDF7F1FF002303600371437161
:10B1D0008360C360012303747047836811B143F037
:10B1E000010301E023F0010383607047836811B11C
:10B1F00043F4807301E023F4807383607047C9B225
:10B2000043680AB1194301E023EA01014160704734
:10B21000836843F00803836070478068C0F3C00010
:10B220007047836843F00403836070478068C0F30D
:10B2300080007047836811B143F4A00301E023F458
:10B24000A003836070478068C0F3805070474368F4
:10B25000013923F4604343EA413343607047436854
:10B2600011B143F4006301E023F4006343607047CD
:10B27000092970B50DD9A1F10A0404EB440407258E
:10B28000A540A340C66826EA050545EA0304C46054
:10B290000BE001EB41040725A54003FA04F406691D
:10B2A00026EA050545EA04030361062A0CD8013A9B
:10B2B00002EB82021F23934001FA02F2446B24EA5C
:10B2C00003031A43426370BD0C2A0CD8073A02EB01
:10B2D00082021F23934001FA02F2046B24EA030363
:10B2E0001A43026370BD0D3A02EB82021F239340A2
:10B2F00001FA02F2C46A24EA03031A43C26270BD6F
:10B30000836811B143F4801301E023F48013836058
:10B310007047C06C80B27047014B1868704700BF1F
:10B320004C240140436811B143F4806301E023F4ED
:10B33000806343607047436811B143F4805301E078
:10B3400023F4805343607047836823F4E043194338
:10B3500081607047836811B143F4004301E023F436
:10B36000004383607047836811B143F4021301E026
:10B3700023F40213836070478068C0F34050704725
:10B38000092970B50DD9A1F10A0404EB440407257D
:10B39000A540A340C66826EA050545EA0304C46043
:10B3A0000BE001EB41040725A54003FA04F406690C
:10B3B00026EA050545EA04030361846B931CC4F384
:10B3C00001555B1BDBB203EB83031F229A409940BC
:10B3D00024EA020444EA0103836370BD836B0139EC
:10B3E00023F4401343EA015383637047425070478C
:10B3F0002831405880B27047436823F4400323F457
:10B40000007319434160704741628262704743682C
:10B4100023F01F03194341607047054B9A6810B130
:10B4200042F4000201E022F400029A60704700BF7B
:10B4300000240140036819420CBF0020012070471E
:10B44000C943016070474368006810EA112004D0C6
:10B45000C9B219420CBF0020012070476FEA1121C8
:10B4600001607047036823F0010303600023036059
:10B4700043608360C3602D4B984234D011D83C3B6D
:10B4800098422AD006D8283B984222D014339842BA
:10B4900021D07047264B984221D01433984220D0B7
:10B4A0007047244B98422DD008D8A3F56773984273
:10B4B0001ED003F5627398421FD070471E4B98420E
:10B4C00029D0143398422BD0283B98422DD11B4BC6
:10B4D0001DE01B4B12E01A4B15E0194B17E0184BFF
:10B4E0001AE0174B1DE0164B5A6842F470021BE03D
:10B4F000134B5A6842F0706216E0104B5A6842F0E3
:10B500000F0211E00D4B5A6842F0F0020CE05A684D
:10B5100042F4706208E0094B5A6842F4704203E05A
:10B52000064B5A6842F470225A6070476C00024021
:10B53000440002401C040240440402400004024053
:10B54000000002408A6810B50C6A036814430A6957
:10B5500023F4FF4314434A6923F0700314438A69B8
:10B560001443CA6914434A6A14438A6A2243134340
:10B570000360CB6843600B6883604B68C36010BD99
:10B580000023036043608360C360036143618361A0
:10B59000C3610362436283627047036811B143F081
:10B5A000010301E023F001030360704703680AB15F
:10B5B000194301E023EA010101607047406880B24D
:10B5C0007047C3004CBF044B044B1B6803420CBFC5
:10B5D00000200120704700BF00040240000002402C
:10B5E000C3004CBF014B024B58607047000402403F
:10B5F00000000240C3004CBF034B044B1B680342D6
:10B600000CBF0020012070470004024000000240EF
:10B61000C3004CBF014B024B58607047000402400E
:10B6200000000240044B00221A605A609A60DA60FF
:10B63000024A5A61704700BF00040140FFFF070043
:10B64000837930B50168027943B3194BCC431D6847
:10B6500002F1804225401D605D6802F582322C4077
:10B660005C6014682143116002689C68D1430C40FF
:10B670009C60DC682140D9604179102906D1996825
:10B6800011439960D9680A43DA6030BD01F1804303
:10B6900003F5823319680A431A6030BD02F1804312
:10B6A00003F582331A6822EA0101196030BD00BF38
:10B6B0000004014000230C22036003714271837176
:10B6C0007047024B1A69104318617047000401402B
:10B6D000034B5B6918420CBF00200120704700BF7C
:10B6E00000040140014B5861704700BF0004014055
:10B6F000054B1A685B69034004D010420CBF002060
:10B70000012070471846704700040140014B586102
:10B71000704700BF00040140044B1A6802F0380271
:10B720001A601A6810431860704700BF002002407A
:10B73000044B1A6822F008021A601A681043186055
:10B74000704700BF00200240044B1A6822F010022C
:10B750001A601A6810431860704700BF002002404A
:10B76000034B044A5A6002F188325A60704700BFA6
:10B770000020024023016745024B1A6942F0800213
:10B780001A61704700200240014BD8698008704759
:10B7900000200240014B186A704700BF00200240A1
:10B7A000024BD869C0F34000704700BF0020024040
:10B7B000024B1868C0F34010704700BF00200240E1
:10B7C000044B1A6909B1104301E022EA0000186134
:10B7D000704700BF002002400128064B03D1D86902
:10B7E00000F001007047DB6818420CBF0020012008
:10B7F000704700BF00200240014BD860704700BF77
:10B8000000200240084BDA68D10709D4DA685207F1
:10B8100008D4DB6813F0100F0CBF0420032070471E
:10B8200001207047022070470020024013B50446F3
:10B83000FFF7E8FF01280FD164B100230193FF2334
:10B840000193019B13B1019B013BF9E7FFF7DAFF7D
:10B85000013CEFE7052002E0002C08BF052002B004
:10B8600010BD38B5054640F6FF70FFF7DFFF04282E
:10B8700014D10B4C40F6FF70236943F0020323619F
:10B880006561236943F040032361FFF7CFFF01287F
:10B8900004D0226941F6FD731340236138BD00BF17
:10B8A0000020024010B540F6FF70FFF7BFFF0428EC
:10B8B00013D10A4C40F6FF70236943F0040323615F
:10B8C000236943F040032361FFF7B0FF012804D050
:10B8D000226941F6FB731340236110BD0020024032
:10B8E00010B540F6FF70FFF7A1FF042829D1154CD1
:10B8F000154B40F6FF70A36003F18833A360236902
:10B9000043F020032361236943F040032361FFF7E1
:10B910008DFF04280ED1226941F6DF7313402361A5
:10B920002369A52243F010032361084B0F201A80DE
:10B93000FFF77CFF012804D0226941F6EF73134022
:10B94000236110BD002002402301674500F8FF1F5E
:10B9500070B505460F200E46FFF768FF042817D183
:10B960000C4C0F20236943F001032361B3B22B80F9
:10B97000FFF75CFF042804D1360C6E800F20FFF720
:10B9800055FF012804D0226941F6FE73134023615C
:10B9900070BD00BF0020024070B505460F200E4666
:10B9A000FFF744FF04280FD1084C0F20236943F010
:10B9B000010323612E80FFF739FF012804D022699B
:10B9C00041F6FE731340236170BD00BF00200240AA
:10B9D00070B505460F200E46FFF728FF042814D146
:10B9E0000A4C0B4B0F20A36003F18833A36023693B
:10B9F00043F0100323612E80FFF718FF012804D0C5
:10BA0000226941F6EF731340236170BD00200240AC
:10BA10002301674510B504460F20FFF707FF0428F0
:10BA20003ED1204B2049E443996001F1883199606F
:10BA30001969E2B241F01001FF2A196104D1C4F37F
:10BA40000723FF2B08D10EE0184B0F201A81FFF7B8
:10BA5000EDFE04281CD1F2E7144A0F205381FFF7B2
:10BA6000E5FE042814D1C4F30743FF2B06D00F4A88
:10BA70000F209381FFF7DAFE042809D1240EFF2C52
:10BA800001D1042006E0094B0F20DC81FFF7CEFE38
:10BA9000012805D0034A41F6EF7311690B40136189
:10BAA00010BD00BF002002402301674500F8FF1FC2
:10BAB00038B5054640F6FF70FFF7B8FE042836D1CA
:10BAC0001B4C1C4B40F6FF70A36003F18833A3604E
:10BAD000236943F020032361236943F0400323617A
:10BAE000FFF7A4FE04281BD1226941F6DF7313403F
:10BAF0002361236943F0100323610F4B0DB1002232
:10BB000000E0A5221A8040F6FF70FFF78FFE0128A3
:10BB10000DD0074A41F6EF7311690B40136138BD30
:10BB2000012804D0226941F6DF731340236138BD38
:10BB3000002002402301674500F8FF1FF8B5114CB3
:10BB4000114B0546A36003F18833A3600F200E4616
:10BB50001746FFF76BFE042813D1236947F0F80757
:10BB600043F0100323613E43084B35435D800F20B3
:10BB7000FFF75CFE012804D0226941F6EF73134001
:10BB80002361F8BD002002402301674500F8FF1F34
:10BB900008B5264B98422FD011D8A3F500639842E0
:10BBA0001ED003F58063984220D0A3F5006398422D
:10BBB0003AD10420012100F0D7FB04202FE01C4BD8
:10BBC00098421FD003F58063984221D0A3F500630B
:10BBD000984229D14020012100F0C6FB40201EE000
:10BBE0000820012100F0C0FB082018E010200121EE
:10BBF00000F0BAFB102012E02020012100F0B4FB7D
:10BC000020200CE08020012100F0AEFB802006E027
:10BC10004FF48070012100F0A7FB4FF480700021E9
:10BC2000BDE8084000F0A0BB08BD00BF0014014003
:10BC3000001C014008B50120014600F095FBBDE85D
:10BC400008400120002100F08FBBCB78F0B5DA0668
:10BC500048BF8A78098803F00F0548BF154311F0E3
:10BC6000FF0F1DD0046800220127974007EA010654
:10BC7000BE4211D197004FF00F0C0CFA07FC05FAE9
:10BC800007F724EA0C04282B44EA070401D1466193
:10BC900002E0482B08BF06610132082AE4D10460A3
:10BCA000FF291FD94468002202F108060127B74086
:10BCB00007EA0106BE4211D197004FF00F0C0CFAB3
:10BCC00007FC05FA07F724EA0C04282B44EA0704CA
:10BCD00001D1466102E0482B08BF06610132082A03
:10BCE000E2D14460F0BD4FF6FF73038002238370FE
:10BCF0000423C3707047836819420CBF00200120E1
:10BD00007047806880B27047C36819420CBF00203A
:10BD100001207047C06880B270470161704741617F
:10BD200070470AB10161704741617047C160704757
:10BD300041F48033836181618361836983697047E2
:10BD4000054B1A6822F07F021204120C114341EADB
:10BD500000101860704700BF00000140014B1860E0
:10BD6000704700BF1C00204230B5134A00F4401554
:10BD7000B5F5401F536884B206D1556823F070634F
:10BD800025F0706555600FE0C20205D5C0F303428F
:10BD9000032505FA02F203E0420D120104FA02F251
:10BDA00023EA020343F0706319B1400D000184409F
:10BDB0002343014A536030BD0000014001F00303FA
:10BDC0009B000F229A40984001F0FC0101F1804154
:10BDD00001F5803110B58C6824EA02028A608A6815
:10BDE00002438A6010BD00BF0B4B6FF070424FF0F2
:10BDF000FF31C3F88010C3F88420C3F88011C3F862
:10BE00008421002202F1C001013200200F2A43F8F0
:10BE10002100F7D1704700BF00E100E0094B4FF06F
:10BE2000206209495A6000229A60D9601A615A61F9
:10BE30009A61DA611A625A624FF0FF329A62DA62EC
:10BE40001A63704700ED00E00000FA0540F0BF60A3
:10BE5000024B40F40030D860704700BF00ED00E0B6
:10BE6000C27830B503785AB31B4A4478D2688578D3
:10BE7000D243C2F30222C2F1040104FA01F10F24F9
:10BE8000D4402C400C4303F00301C9002401FF22DD
:10BE90008C408A4003F0FC0303F1604303F56143E7
:10BEA000D3F8005325EA020122400A43C3F80023D5
:10BEB00003780122590903F01F0302FA03F306E095
:10BEC0005909012203F01F0302FA03F32031034A48
:10BED00042F8213030BD00BF00ED00E000E100E09D
:10BEE0000023037043708370C3707047F8F735B94F
:10BEF000F8F735B9F8F735B9F8F735B90001F8F7BB
:10BF000034B9F8F735B9024B5868C0F309307047B7
:10BF100000ED00E000F01F03012202FA03F34009E4
:10BF2000044A403052F820001840C31A5842584181
:10BF3000704700BF00E100E0014B1860704700BF90
:10BF400000EF00E04209012300F01F0003FA00F0B7
:10BF5000024B603243F82200704700BF00E100E06E
:10BF6000024B5868C0F30900704700BF00ED00E0C5
:10BF700000F01F03012202FA03F34009044A803053
:10BF800052F820001840C31A58425841704700BF69
:10BF900000E100E0014B1868704700BF00ED00E0D1
:10BFA00021F0604121F07F01014B08439860704708
:10BFB00000ED00E0014A024BDA6070470400FA0528
:10BFC00000ED00E0014A024BDA6070470100FA051B
:10BFD00000ED00E0044B1A6909B1104301E022EAC8
:10BFE00000001861704700BF00ED00E0012300F081
:10BFF0001F0003FA00F0044B5A6A09B1104301E034
:10C0000022EA00005862704700ED00E0114B30B5A5
:10C01000DB68DB43C3F30223C3F10404A140FF2424
:10C0200024FA03F31A401143C0F30122D2009440D2
:10C03000090101FA02F2C0F38110800000F16040B2
:10C0400000F56D40836923EA0404846185692A430D
:10C05000826130BD00ED00E0C0F383200123834006
:10C06000034A506A1840C31A58425841704700BFEB
:10C0700000ED00E000F01F00012101FA00F0024B8A
:10C080005A6802435A60704700ED00E000F01F005C
:10C09000411E012000FA01F1024B5A680A435A601E
:10C0A000704700BF00ED00E0C0F383300123834000
:10C0B000034A506A1840C31A58425841704700BF9B
:10C0C00000ED00E0C0F38142094B0AB9D86A70471D
:10C0D000012A0AD1C0F30152986AD300D840022A3B
:10C0E00014BF00F00F00C0B27047186B704700BF5C
:10C0F00000ED00E0034B10F4800F0CBF586B986B01
:10C10000704700BF00ED00E00C4B1A6842F00102DE
:10C110001A6059680A4A0A405A601A6822F0847202
:10C1200022F480321A601A6822F480221A605A6857
:10C1300022F4FE025A6000229A607047001002400A
:10C140000000FFF80C4BB0F5803F1A6822F48032F3
:10C150001A601A6822F480221A6003D0B0F5802F8A
:10C1600004D070471A6842F4803202E01A6842F440
:10C17000A0221A60704700BF00100240034B1A68EB
:10C1800022F0F80242EAC000186070470010024036
:10C19000014B1860704700BF00004242034B5A68D1
:10C1A00022F47C121143084358607047001002408B
:10C1B000014B1860704700BF60004242034B5A6851
:10C1C00022F0030210435860704700BF0010024085
:10C1D000024B586800F00C00704700BF001002408E
:10C1E000034B5A6822F0F00210435860704700BFBA
:10C1F00000100240034B5A6822F4E062104358607A
:10C20000704700BF00100240034B5A6822F460528E
:10C2100042EAC0005860704700100240044B1A7890
:10C2200009B1104301E022EA00001870704700BF16
:10C2300009100240014B1860704700BFD80042420D
:10C24000034B5A6822F4404210435860704700BFC5
:10C2500000100240064B002201281A701A7002D00A
:10C26000042802D070471870704705221A70704772
:10C2700020100240014B1860704700BF800442420A
:10C28000024B1A6A10431862704700BF0010024048
:10C29000014B1860704700BF3C0442421C4B10B574
:10C2A0005A6802F00C02042A01D0082A01D0194A67
:10C2B0000EE05A685968C2F38342CC0302F10202CD
:10C2C00002D55968890301D5134900E011494A4351
:10C2D00002605968114AC1F30311545C0168E140DE
:10C2E00041605C68C4F30224145D21FA04F48460A4
:10C2F0005C68C4F3C224145DE140C1605B68C3F3B1
:10C3000081331A44137CB1FBF3F1016110BD00BF0E
:10C310000010024000127A0000093D00E506010805
:10C32000044B5A6909B1104301E022EA0000586148
:10C33000704700BF00100240044B9A6909B11043D6
:10C3400001E022EA00009861704700BF001002403F
:10C35000044BDA6909B1104301E022EA0000D86118
:10C36000704700BF00100240044BDA6809B1104367
:10C3700001E022EA0000D860704700BF00100240D0
:10C38000044B1A6909B1104301E022EA0000186168
:10C39000704700BF00100240014B1860704700BF9B
:10C3A00040044242014B1860704700BF4C004242BB
:10C3B000014B1870704700BF071002404309012B62
:10C3C000074A01D1136803E0022B0CBF136A536ABA
:10C3D00000F01F0023FA00F000F00100704700BFDA
:10C3E0000010024008B53120FFF7E8FF094B187034
:10C3F0005A6801325A601A7822B95A6840F2FF131B
:10C400009A42F0D13120FFF7D9FF003018BF012048
:10C4100008BD00BFBC090020024B5A6A42F080727E
:10C420005A62704700100240034B9B6818420CBFD1
:10C4300000200120704700BF00100240014B18701F
:10C44000704700BF0A10024008B5164B98421BD037
:10C4500003F5744398420BD0A3F5784398421FD15B
:10C460004FF480400121FFF78BFF4FF4804012E032
:10C470004FF480500121FFF777FFBDE808404FF4EB
:10C4800080500021FFF770BF4FF400400121FFF7FB
:10C4900077FF4FF400400021BDE80840FFF770BF70
:10C4A00008BD00BF003C00400B8810B54C880288D6
:10C4B00023438C8802F441522343CC8823430C89C4
:10C4C00023434C8923438C892343CC89234313433F
:10C4D0009BB20380838B23F400631B041B0C8383B8
:10C4E0000B8A038210BD838BF0B523F47B6323F0AA
:10C4F0000F031B041B0C8383022303840B89868B8D
:10C50000022B87B005460C46B6B223D08B8801A813
:10C51000002B14BF02270127FFF7C0FEE388228902
:10C52000B3F5007F019B4FF00A011CBF7F017A43E6
:10C5300001FB03F308BF1202B3FBF2F305330A2237
:10C540009BB2B3FBF2F303F001021202C3F34F03F9
:10C5500092B200E00022991E89B2FE2928BF002273
:10C56000E18828BF022313430B439BB22B8423880B
:10C570006288334343F400631343A2881343628900
:10C5800013439BB2AB8307B0F0BD0023038043800D
:10C590008380C380038143818381C3810723038216
:10C5A000704700230222038043808380C38002817E
:10C5B00043817047038819B19BB243F0400303E005
:10C5C00023F040031B041B0C03807047838B19B1BD
:10C5D0009BB243F4806303E023F480631B041B0CD1
:10C5E00083837047090901238B409BB21AB182886B
:10C5F00092B2134303E0828892B222EA030383805B
:10C60000704783889BB20AB1194301E023EA010114
:10C610008180704781817047808980B270474FF672
:10C62000FF639942038803D09BB243F4807303E015
:10C6300023F480731B041B0C03807047838819B19B
:10C640009BB243F0040303E023F004031B041B0C20
:10C6500083807047038823F400631B041B0C038052
:10C6600003889BB219430180704703889BB243F44F
:10C67000805303807047038819B19BB243F4005381
:10C6800003E023F400531B041B0C038070470129B3
:10C6900014BF008B808A80B27047008A80B27047D6
:10C6A000B1F5804F038803D19BB243F4804303E08C
:10C6B00023F480431B041B0C038070470389194239
:10C6C0000CBF002001207047202906D10389038870
:10C6D0009BB243F0400303807047402901D00829F2
:10C6E00001D103897047C94389B20181704701F0C4
:10C6F0000F02012303FA02F210B584880089A4B264
:10C7000080B2104005D009098B401C420CBF0020AC
:10C71000012010BD552906D1038903889BB243F03F
:10C72000400303807047562901D0532901D1038962
:10C73000704701F00F01012303FA01F1C94389B2E7
:10C7400001817047044B04281A680CBF42F00402B0
:10C7500022F004021A60704710E000E0014B5860BC
:10C76000704700BF10E000E00128084B03D11A68B1
:10C7700042F0010204E0023004D11A6822F0010202
:10C780001A60704700229A60704700BF10E000E016
:10C79000044B1A6810B142F0020201E022F00202DA
:10C7A0001A60704710E000E0014B9868704700BFC6
:10C7B00010E000E0C308022B044B0CBF1B68DB68D1
:10C7C00023FA00F000F00100704700BF10E000E025
:10C7D00030B5048C24F001042404240C0484058B5B
:10C7E000048CADB225F0F305A4B22A4324F0020470
:10C7F00042EA031344F001049DB2214305830184FE
:10C8000030BD30B5048C24F010042404240C0484BE
:10C81000058B048C25F44075A4B22D052D0D24F054
:10C82000200444F0100445EA022242EA033344EAB9
:10C8300001119BB28CB20383048430BD08B52E4B2A
:10C8400098423AD010D8A3F50063984225D003F55A
:10C85000806398422BD0B0F1804F4CD1012001462B
:10C86000FFF78EFD01201DE0244B984231D004D803
:10C87000A3F58063984226D008BD214B984204D08E
:10C8800003F5006398422AD008BD4FF400600121EF
:10C89000FFF76AFD4FF4006028E002200121FFF756
:10C8A0006FFD02200021BDE80840FFF769BD0420AC
:10C8B0000121FFF765FD0420F4E708200121FFF7BF
:10C8C0005FFD0820EEE710200121FFF759FD102041
:10C8D000E8E720200121FFF753FD2020E2E74FF495
:10C8E00000500121FFF740FD4FF400500021BDE84A
:10C8F0000840FFF739BD08BD000C0040001400409F
:10C90000002C01400388CA8803F08F03038003884A
:10C910009BB213434A8813439BB203808B88838561
:10C920000B880385054B984203D003F500639842BA
:10C9300001D10B7A0386012383827047002C0140CA
:10C94000038C70B523F001031B041B0C0384038CC0
:10C950008488028B0D8822F070021204120C4E881B
:10C960002A430D8923F002031B043543ADB21B0C8F
:10C970002B43CD88A4B285860D4DA84203D005F582
:10C980000065A8420FD14D8923F008032B438D8801
:10C9900023F004032B4347F6FF452540CC898989C2
:10C9A0000C43A4B22C4384800283038470BD00BF77
:10C9B000002C0140038C30B523F010031B041B0C2A
:10C9C0000384038C8288048B0D8824F4E0442404BF
:10C9D000240C23F0200344EA05241B040D891B0CBE
:10C9E00043EA05134D8892B243EA0513CD88A4B2F9
:10C9F0000587114D9BB2A84203D005F50065A842FA
:10CA000016D14D8923F080039BB243EA05134FF6FC
:10CA1000BF751D408B8845EA031347F2FF3515406B
:10CA20008A899BB245EA8205CA8945EA820292B2A6
:10CA300082800483038430BD002C0140038C30B518
:10CA400023F480731B041B0C0384038C8288848B67
:10CA50000D8824F070042404240C23F400732C4368
:10CA60001B040D891B0C43EA05234D8892B243EA4F
:10CA70000523CD889BB28587104DA84203D005F5CC
:10CA80000065A84216D14D8923F400639BB243EAA6
:10CA900005234FF6FF351D408B8845EA032344F6F6
:10CAA000FF7515408A899BB245EA0215CA8945EA95
:10CAB000021292B282808483038430BD002C014034
:10CAC000038C30B523F480531B041B0C0384038CAC
:10CAD0008488828B0D8822F4E0421204120C23F425
:10CAE000005342EA05221B040D891B0C43EA05335F
:10CAF0004D88A4B243EA0533CD8892B2A0F84050E5
:10CB0000084D9BB2A84203D005F50065A84205D1A7
:10CB10008989C4F30D0444EA8114A4B28480828319
:10CB2000038430BD002C01404A880B8813438A8857
:10CB30001343CA8813430A8913434A8913438A89D2
:10CB400013439BB2A0F8443070474FF6FF738380C5
:10CB500000230380C3804380037270470023038057
:10CB600043808380C380038143818381C381704775
:10CB700000230122038043808280C38003817047A9
:10CB80000023038043808380C380038143818381AA
:10CB90007047038819B19BB243F0010303E023F00F
:10CBA00001039B059B0D03807047B0F8443029B109
:10CBB0006FEA43436FEA53439BB201E0C3F30E03B2
:10CBC000A0F84430704783899BB20AB1194301E051
:10CBD00023EA010181817047818270470A43A0F8EE
:10CBE0004820704783899BB20AB1194301E023EAC8
:10CBF000010181817047038923F007031B041B0C8B
:10CC000003817047038923F070031B041B0C194335
:10CC1000018103899BB243F007030381704738B554
:10CC20000D46602D114604464FF0010202D1FFF778
:10CC3000E8FD01E0FFF7CCFD238923F070031B041E
:10CC40001B0C2B43238123899BB243F007032381D1
:10CC500038BD10B5048942EA0323E4B21C43A4B2F0
:10CC60002143018110BD10B50446FFF7F2FF23896F
:10CC700023F077031B041B0C43F07703238110BDC3
:10CC800010B50446FFF7E5FF23899BB243F48043C8
:10CC9000238110BD018582827047038823F07003D1
:10CCA0009B059B0D194301807047038923F0700396
:10CCB0001B041B0C19430181704770B50589048B57
:10CCC000068C24F44074B6B224F0030426F0220645
:10CCD00025F00705240432432D04240C2D0C44F4C4
:10CCE000807442EA0313294344F001049EB2018197
:10CCF0000483068470BD038B23F070031B041B0C9C
:10CD0000194301837047038B23F4E0431B041B0C7E
:10CD100043EA01218BB203837047838B23F07003B6
:10CD20001B041B0C194381837047838B23F4E0435E
:10CD30001B041B0C43EA01218BB2838370470388D9
:10CD400019B19BB243F0800303E023F080039B05FD
:10CD50009B0D03807047838819B19BB243F0040395
:10CD600003E023F004031B041B0C838070478388BB
:10CD700019B19BB243F0080303E023F008031B043E
:10CD80001B0C83807047838819B19BB243F0010369
:10CD900003E023F001031B041B0C83807047038B0B
:10CDA00023F008031B041B0C194301837047038BFA
:10CDB00023F400631B041B0C43EA01218BB20383A1
:10CDC0007047838B23F008031B041B0C19438183DA
:10CDD0007047838B23F400631B041B0C43EA01217F
:10CDE0008BB283837047038B23F004031B041B0C5B
:10CDF000194301837047038B23F480631B041B0CCE
:10CE000043EA01218BB203837047838B23F0040331
:10CE10001B041B0C194381837047838B23F48063AD
:10CE20001B041B0C43EA01218BB283837047038BE5
:10CE300023F080031B041B0C194301837047038BF1
:10CE4000C3F30E0343EA01218BB203837047838B44
:10CE500023F080031B041B0C194381837047838BD1
:10CE6000C3F30E0343EA01218BB283837047038C23
:10CE700023F002031B041B0C194301847047038C2D
:10CE800023F008031B041B0C194301847047038C17
:10CE900023F020031B041B0C43EA01118BB2038413
:10CEA0007047038C23F080031B041B0C43EA011121
:10CEB0008BB203847047038C23F400731B041B0C98
:10CEC00043EA01218BB203847047038C23F400638F
:10CED0001B041B0C43EA01218BB203847047038CB3
:10CEE00023F400531B041B0C43EA01318BB203846F
:10CEF000704701238B408A4010B5048CA4B224EA09
:10CF000003030384038C13439BB2038410BD0423E7
:10CF10008B408A4010B5048CA4B224EA0303038436
:10CF2000038C13439BB2038410BD01238B4010B5C7
:10CF3000048C1830A4B224EA0303038121F008030F
:10CF40003BB9490844584FF68F7323404350435828
:10CF50000AE00439C1F34E01445848F6FF732340F8
:10CF600043501202435892B21A43425010BD0388F4
:10CF700019B19BB243F0020303E023F002039B05C7
:10CF80009B0D03807047038819B19BB243F00403E3
:10CF900003E023F004039B059B0D03807047838807
:10CFA00019B19BB243F0800303E023F080031B041C
:10CFB0001B0C83807047038823F008039B059B0D9F
:10CFC000038003889BB2194301807047838823F054
:10CFD00070031B041B0C838083889BB219438180E0
:10CFE0007047038923F007031B041B0C038103898B
:10CFF0009BB2194301817047038923F080031B040E
:10D000001B0C038103899BB2194301817047818402
:10D010007047818570478186704701877047818797
:10D020007047A0F840107047038B23F00C031B04DB
:10D030001B0C0383038B9BB2194301837047038B43
:10D0400023F440631B041B0C0383038B9BB243EA52
:10D0500001218BB203837047F8B50C464988A2883A
:10D060000029B4F800E014BF00270227012A054672
:10D0700014BF012602262389BEF1000F11D1FFF74C
:10D08000A7FB2846E188FFF7CFFF284639463246FE
:10D090002389FFF7B6FB2846E188BDE8F840FFF793
:10D0A000CEBFFFF7AEFB2846E188FFF7C8FF284652
:10D0B000394632462389FFF78BFB2846E188BDE8D5
:10D0C000F840FFF7B1BF838B23F00C031B041B0C4C
:10D0D0008383838B9BB2194381837047838B23F4B3
:10D0E00040631B041B0C8383838B9BB243EA0121A7
:10D0F0008BB283837047F8B50E880D460446498885
:10D10000AA882B893EB9FFF763FB2046E988BDE872
:10D11000F840FFF789BF042E07D1FFF772FB2046C6
:10D12000E988BDE8F840FFF78ABF082EEF88068C33
:10D130001CD126F480763604360C0684858B068C4A
:10D14000ADB225F0F30545EA0313B6B29BB21A431C
:10D1500026F4007343EA012189B241F4807182838D
:10D1600001843946BDE8F840FFF7ADBF26F480568C
:10D170003604360C0684858B068C25F440752D0507
:10D18000B6B22D0D45EA022526F4005242EA0131DD
:10D1900045EA033389B29BB241F480518383018411
:10D1A0003946BDE8F840FFF799BF0388DBB203803A
:10D1B00003889BB2194301807047808E80B270470C
:10D1C000008F80B27047808F80B27047B0F8400007
:10D1D00080B27047808C80B27047008D80B27047FB
:10D1E000038A19420CBF002001207047C94389B24D
:10D1F00001827047038A828911EA030092B203D048
:10D2000011420CBF002001207047C94389B201823E
:10D21000704700BF08B5224B98422CD008D8A3F520
:10D220000063984217D003F5806398421BD008BD75
:10D230001C4B984227D003F5684398422FD14FF4F6
:10D2400080400121FFF790F8BDE808404FF480408E
:10D250000021FFF789B84FF400300121FFF790F863
:10D260004FF4003016E04FF480200121FFF788F8DA
:10D270004FF480200EE04FF400200121FFF780F8EA
:10D280004FF4002006E04FF480100121FFF778F8FA
:10D290004FF480100021BDE80840FFF771B808BDC9
:10D2A000004C004000500040038ACA889BB223F41F
:10D2B0004053134330B503820D4682890989AB88F8
:10D2C00092B20B43698922F4B0520B4322F00C0254
:10D2D00013439BB28381838AAA899BB223F4407350
:10D2E00087B013430446838201A8FEF7D7FF049A50
:10D2F000039B0E498C4208BF134619214B432A68F1
:10D300009200B3FBF2F16423B1FBF3F212011009B6
:10D3100003FB101109013231B1FBF3F303F00F03EA
:10D320001A4392B2228107B030BD00BF00380140DD
:10D330004FF4165303600C2200238380C3800381C3
:10D340004281838170470B8810B54C88028A234341
:10D350008C88C98892B223430B4322F47062134332
:10D360009BB2038210BD0023038043808380C3806F
:10D370007047838919B19BB243F4005303E023F44F
:10D3800000531B041B0C83817047C1F3421310B57B
:10D39000012401F01F01A34204FA01F101D10C3074
:10D3A00003E0022B0CBF1030143003680AB119439C
:10D3B00001E023EA0101016010BD838A9BB20AB13A
:10D3C000194301E023EA010181827047038A23F0B7
:10D3D0000F031B041B0C0382038A9BB219430182B7
:10D3E0007047838923F400631B041B0C83818389AA
:10D3F0009BB2194381817047838919B19BB243F075
:10D40000020303E023F002031B041B0C838170471B
:10D41000038A23F020031B041B0C0382038A9BB2A4
:10D42000194301827047038A19B19BB243F48043C8
:10D4300003E023F480431B041B0C03827047C1F3F9
:10D440000801818070478088C0F308007047838995
:10D450009BB243F0010383817047038BDBB20383EC
:10D46000038B9BB243EA012101837047038B03F4D2
:10D470007F430383038B9BB2194301837047838AE5
:10D4800019B19BB243F0200303E023F020031B04F7
:10D490001B0C83827047838A19B19BB243F010033F
:10D4A00003E023F010031B041B0C83827047838A64
:10D4B00019B19BB243F0080303E023F008031B04F7
:10D4C0001B0C83827047838A23F004031B041B0C0C
:10D4D0008382838A9BB2194381827047838A19B100
:10D4E0009BB243F0020303E023F002031B041B0C76
:10D4F00083827047038819420CBF002001207047C7
:10D50000C94389B20180704710B5C1F3421401F0DC
:10D510001F030122012C02FA03F201D1838903E0E7
:10D52000022C0CBF038A838A9BB21340028892B2FA
:10D5300043B10123090A03FA01F111420CBF002093
:10D54000012010BD184610BD090A01238B40DB43A2
:10D550009BB20380704700BF684620F007018D46EC
:10D5600001B500230B4A0C499818884204D20B4994
:10D57000595899500433F5E7094B0A4A934203D2AC
:10D58000002243F8042BF8E702F0A4FBBDE80140B9
:10D590008546704700000020640500203C08010813
:10D5A000680500204410002010B5064C18B9236807
:10D5B00001221A8210BD044B1B681B689847206823
:10D5C0000A3010BDE00F00209C0F002010B5064C63
:10D5D00018B9236801221A8210BD044B1B689B688E
:10D5E000984720680C3010BDE00F00209C0F0020F1
:10D5F00010B5204B18B91B6802221A8210BD1E4AB2
:10D600001968002010800C78134614F07F040DD1A7
:10D610004A7A910644BF0221197012F0400F1A781D
:10D6200014BF22F0010242F0010214E0012C1FD0CD
:10D63000022C1ED1497901F00F02920002F18042C2
:10D6400002F5B84211F0800F126806D002F03002E5
:10D65000102A07D101221A7004E002F44052B2F5F8
:10D66000805FF6E7054B1B681B699847024810BDB1
:10D67000104610BDE00F00203C1000209C0F002041
:10D68000234A2DE9F84314689046238A267A214FCD
:10D69000A3B9042E12D120490A78012A0AD11F4ABF
:10D6A00010681F4A80B202445200136030223A8050
:10D6B0000B7027E010233B80072623E0A58AAB42AE
:10D6C0008CBF022604269D4228BF1D462846A3691A
:10D6D00098478146002000F06BFE2A4601464846E6
:10D6E00000F06EFC2946002000F07EFE238A4FF4F5
:10D6F00040525B1B2382638A1D4430233B80094BCD
:10D7000065821A80D8F800301E72BDE8F88300BF29
:10D71000E00F002040100020C4090020505C0040B1
:10D72000023000203E10002010B50A4B0A491B6849
:10D730004978DA7891420AD3997841B99C8834B90A
:10D740009A72064B1B685B689847204610BD022002
:10D7500010BD00BFE00F0020D80000209C0F00206B
:10D7600038B50E4A0E4C1268236892695879D978F8
:10D77000904723689A7A7AB170B91A7962B99D781C
:10D7800055B9084B1B68DB689847236828465A79C7
:10D79000DA72DA781A7338BD022038BD780F0020AB
:10D7A000E00F00209C0F002038B52F4B1B68187825
:10D7B00010F07F0004D15A7A22F020025A7238BD4C
:10D7C00002284ED15A88002A4CD11A79002A49D110
:10D7D0005A79264D22F08000840004F1804101F541
:10D7E000B84109682D7812F0800F14BF01F03001A4
:10D7F00001F44051A84234D2002932D09B7A83B33D
:10D8000004F1804404F5B844120623680CD503F0F3
:10D810003003102B1FD1C4B2204600F080FD2046FB
:10D82000302100F055FC16E003F44053B3F5805F5F
:10D8300011D128B90E4B93F82C1000F0F6FD01E041
:10D8400000F05DFD236823F4804323F070039BB256
:10D8500083F440532360074B1B685B6998470020A3
:10D8600038BD022038BD00BFE00F0020D8000020E6
:10D87000500000209C0F002038B51D4B1D4D19682D
:10D880002D784A7922F08004A30003F1804000F54E
:10D89000B840006812F0800F14BF00F0300000F4B0
:10D8A0004050AC4222D24C8804BBF8B1897AE9B12D
:10D8B00003F1804303F5B84312F0800F1A6807D0D4
:10D8C00022F4E04222F0400292B282F0100206E01E
:10D8D00022F4804222F0700292B282F480521A60E6
:10D8E000054B1B689B699847002038BD022038BD56
:10D8F000E00F0020D80000209C0F002008B5064B48
:10D900001B685A7A42F020025A72044B1B68DB698A
:10D910009847002008BD00BFE00F00209C0F0020AA
:10D92000054B1A68538A18B98988CB1A1382704735
:10D9300008681844704700BFE00F002008B50B4B83
:10D94000002093F82C1000F070FD094B1B68187A2A
:10D95000082806D1074B4FF480521A80064B10223C
:10D960001A80B0F109035842584108BD5000002008
:10D97000E00F00203E10002040100020F7B5914F2E
:10D98000914B3A68914D92B213442E685B001C682B
:10D99000337A092B15D0A4B2640004F1804404F555
:10D9A000C0442378337063787370A08800F0E8FE79
:10D9B000708020892E6800F0E3FEB080A2892B6879
:10D9C000DA802B6801221A72DA885C78002A61D129
:10D9D0001A7812F07F023AD1092C02D1FFF7A4FE87
:10D9E00044E0052C0FD193F90320002A01DA082323
:10D9F0004DE09A78002AFAD19A88002AF7D19B7ACA
:10DA0000002B37D0F3E7032C13D1DA78012A07D0A3
:10DA10006F4B20461B685B699847032828D135E087
:10DA20009A88002AF4D15B7A9806F1D5FFF766FF51
:10DA30001CE0012CECD1DA78012AE9D19A88002A7D
:10DA4000E6D15B7A9906E3D5FFF7AEFE0EE0012A38
:10DA500004D10B2CDCD1FFF783FE07E0022AD7D1DB
:10DA6000012CF1D0032CD3D1FFF706FF10B1CFE783
:10DA70000028BCD13A68574B92B213445B00002295
:10DA80001A60554B30221A80062300E009232A68C9
:10DA90001372D0E0062C13D11A78520678D19A78F6
:10DAA0004B4B012A02D11B68DB6968E0022A02D1D4
:10DAB0001B681B6A63E0032A6AD11B685B6A5EE02D
:10DAC000002C3DD15988002962D15A6822F47F4246
:10DAD000B2F5003F5CD11A7812F07F0204D19B8826
:10DAE000002B00F0AC8053E0012A0DD1384A587960
:10DAF00012689269904700284AD1344B1B689B7A80
:10DB0000002B40F09C8043E0022A41D15B793348EE
:10DB100003F00F018A0002F1804202F5B842126858
:10DB2000007813F0800F14BF02F0300202F440526C
:10DB300081422DD213F0700F2AD1002A7FD127E025
:10DB4000082C03D11B785B067BD021E00A2C1FD167
:10DB50001A7802F07F02012A1AD19A7AC2B1598842
:10DB6000B1B95A6822F47F42B2F5803F10D1184A09
:10DB70005879126892699047002864D008E03BB158
:10DB80002A680024548293612046984720460AE080
:10DB90000F4B1A682B68126958789047032802D1F6
:10DBA0000A4B1B6805E02B684FF6FF711A8A8A4200
:10DBB00001D1092203E0022800D08AB908221A7292
:10DBC00039E000BF505C004004300020E00F00202E
:10DBD000780F00200230002040100020D8000020E4
:10DBE00093F90010002920DAD98801910198824226
:10DBF000164802D9019A1A8210E08A420ED20168B0
:10DC000091F82C108A4201D2002105E092FBF1F438
:10DC100001FB142212B901210D4A1170026892F819
:10DC20002C209A82FFF72CFD05E003221A72094B83
:10DC30004FF440521A80FFF781FE03B0F0BD064B4F
:10DC40009EE7064B9CE7064B9AE700BF780F002043
:10DC5000C40900203E100020F1D50008A9D5000815
:10DC6000CDD50008F8B52B4D2C68237A032B01D0B5
:10DC7000052B41D1A369228AABB1A2B1A68A9642F3
:10DC800028BF164630469847238A07469B1B2382A7
:10DC9000638A00203344638200F098FB32460146D9
:10DCA000384600F0A5F9238A53B11B4B00204FF4EE
:10DCB000405201461A8000F097FB184B30221A8020
:10DCC000238AA28A9A4202D82B68032202E01BB15F
:10DCD0002B6805221A720CE02A6806211172104A7C
:10DCE0001168104A89B20A44520013600B4B30226B
:10DCF0001A802B681B7A06E0072B03D10A4B1B689E
:10DD0000DB68984708232A681372BDE8F840FFF7DC
:10DD100015BE00BFE00F00203E1000204010002084
:10DD2000505C004002300020780F002030B50B4BD3
:10DD30001C780023A3420CD203F1805202F5B852A2
:10DD400091000D6848F68F722A401A430A60013329
:10DD5000F0E7034B40F08000186030BDD800002091
:10DD60004C5C004010B5134C23681A7A022A01D08B
:10DD7000042A04D1FFF784FC23681B7A13E0062AE7
:10DD800010D15A78052A09D11A78520606D1D878C6
:10DD9000FFF7CCFF084B1B681B6A9847074B1B68B3
:10DDA0009B689847082322681372BDE81040FFF76C
:10DDB000C5BD00BFE00F00209C0F0020780F0020A1
:10DDC000704700BF08B5074A074B08491360022295
:10DDD0001A72074B074A1360074A1B68116098477D
:10DDE00008BD00BFE00F0020800F0020B40000201D
:10DDF00050000020780F00209C0F002070B54C4A86
:10DE00004C4B116888B20C04188040F1908047F6A2
:10DE1000FF7111601A88484C02F00F022270002A2C
:10DE20005FD1464C464D2268464E02F440522A804D
:10DE3000226802F030023280226822F4804222F00E
:10DE4000700292B282F400522260226822F4E04210
:10DE500022F0400292B282F0200222601B88D80693
:10DE600002D52368190607D5226848F60F731340B8
:10DE70002360FFF777FF12E01A0507D5226840F606
:10DE80008F7313402360FFF779FD08E01804B6D5BF
:10DE9000226840F68F7313402360FFF7E3FE236888
:10DEA0002A8823F4804323F070039BB2D10448BF37
:10DEB00083F480539504214A48BF83F400531360D0
:10DEC0001368318823F4E04323F040039BB2CC066F
:10DED00048BF83F01003880648BF83F02003136017
:10DEE00070BD930003F1804303F5B8431D68290416
:10DEF00009D5186840F68F7101401960124B013A3C
:10DF000053F8223098472B067FF579AF217848F6F1
:10DF10000F728B0003F1804303F5B8431868013991
:10DF200002401A60094B53F82130984767E770BDEB
:10DF3000445C0040760F00207C0F0020005C004015
:10DF40003E10002040100020DC000020F8000020DF
:10DF500008B5164A164B116888B20904188024D5F2
:10DF600047F6FF7111601A88124B02F00F021A7007
:10DF7000930003F1804303F5B8431968080407D5FB
:10DF8000186840F68F7101401960013A0A4B08E0A9
:10DF90000906DED5186848F60F7101401960074B75
:10DFA000013A53F822309847D3E708BD445C00405B
:10DFB000760F00207C0F0020DC000020F8000020FD
:10DFC00030B501F10051013201F5405152104900C4
:10DFD0000023934200F1020009D010F8015C10F810
:10DFE000024C44EA052421F823400133F1E730BD17
:10DFF00010B501F10051013201F5405152104900B4
:10E000000023934205D051F8234020F813400133F8
:10E01000F7E710BD014B1860704700BF405C00403F
:10E02000014B186880B27047405C0040014B18609B
:10E03000704700BF445C0040014B186880B27047D5
:10E04000445C0040014B186880B27047485C004057
:10E05000014B1860704700BF4C5C0040014B1868D2
:10E0600080B270474C5C00404FF6F873014A0340A1
:10E0700013607047505C0040014B186880B27047D5
:10E08000505C0040800000F1804000F5B840016025
:10E090007047800000F1804000F5B840006880B211
:10E0A0007047800000F1804000F5B840036823F419
:10E0B000EC4323F0700319438BB203607047800078
:10E0C00000F1804000F5B840006800F4C06070477F
:10E0D000800000F1804000F5B8400368CA0623F4D0
:10E0E000E04323F040039BB248BF83F010038A064D
:10E0F00048BF83F0200303607047800000F1804038
:10E1000000F5B8400368CA0423F4804323F0700389
:10E110009BB248BF83F480538A0448BF83F4005302
:10E1200003607047800000F1804000F5B84001298D
:10E13000026802D14EF6FF7303E0022903D14FF6C5
:10E14000EF73134003607047800000F1804000F5DA
:10E15000B840006800F030007047800000F1804057
:10E1600000F5B840006800F440507047800000F1AE
:10E17000804000F5B840036823F4E04323F04003F7
:10E180009BB283F0300303607047800000F1804051
:10E1900000F5B840036823F4804323F070039BB27A
:10E1A00083F4405303607047800000F1804000F525
:10E1B000B840036823F4E04323F0700343F4807312
:10E1C0009BB203607047800000F1804000F5B840CA
:10E1D000036823F4E24323F070031B041B0C036069
:10E1E0007047800000F1804000F5B840036823F4D8
:10E1F000E24323F070031B041B0C03607047800094
:10E2000000F1804000F5B840036823F4E04323F0B8
:10E21000700343F480739BB203607047800000F189
:10E22000804000F5B840036823F4E04323F0700316
:10E2300043F480739BB203607047800000F180401C
:10E2400000F5B840036823F4E24323F070031B0495
:10E250001B0C03607047800000F1804000F5B8405F
:10E26000006800F03000B0F1100358425841704788
:10E27000800000F1804000F5B840006800F4405094
:10E28000B0F58053584258417047800000F18040FB
:10E2900000F5B840036823F070031B051B0D0360F5
:10E2A0007047800000F1804000F5B840036823F417
:10E2B000E14323F070031B041B0C036070478000D4
:10E2C00000F1804000F5B840036823F4E04323F0F8
:10E2D00070031B041B0C43F48043036070478000F1
:10E2E00000F1804000F5B840036823F4E04323F0D8
:10E2F00070031B041B0C43F0400303607047800055
:10E3000000F1804000F5B84003685B0406D5026860
:10E3100048F68F73134043F48043036070478000D6
:10E3200000F1804000F5B84003685B0606D502683E
:10E3300048F68F73134043F040030360704780003A
:10E3400000F1804000F5B840036823F4E04323F077
:10E3500070031B041B0C194301607047800000F11F
:10E36000804000F5B840006800F00F007047074B90
:10E3700049081B6849009BB203EBC00000F1005044
:10E3800000F5405040000160704700BF505C004005
:10E39000054B49081B6849009BB203EBC000034BC7
:10E3A00003445B0019607047505C0040043000205B
:10E3B000054B1B689BB203EBC00000F1005000F559
:10E3C0004050400000887047505C0040044B1B6880
:10E3D0009BB203EBC000034B03445B0018887047FB
:10E3E000505C004004300020044B1B689BB203EBE0
:10E3F000C000034B03445B0019607047505C004051
:10E40000023000203E2909D94B09C90604BF03F197
:10E41000FF339BB29B0243F4004304E04B08CA075E
:10E4200048BF01339B02036070470E4B3E291B68B7
:10E430009BB203EBC0000C4B03444FEA430209D9E3
:10E440004B09C80604BF03F1FF339BB29B0243F4A0
:10E45000004304E04B08C90748BF01339B02136027
:10E46000704700BF505C004006300020054B1B6821
:10E470009BB203EBC000044B03445B001868C0F37D
:10E4800009007047505C004002300020054B1B68BB
:10E490009BB203EBC000044B03445B001868C0F35D
:10E4A00009007047505C00400630002010B50B4C4E
:10E4B000C000236849089BB2034403F1005303F5ED
:10E4C00040535B0049001960236852089BB218440E
:10E4D000034B520003445B001A6010BD505C0040C7
:10E4E00004300020064B49081B6849009BB203EB2F
:10E4F000C00000F1005000F540504000016070473E
:10E50000505C0040054B49081B6849009BB203EB77
:10E51000C000034B03445B0019607047505C00402F
:10E5200004300020054B1B689BB203EBC00000F1D8
:10E53000005000F54050400000887047505C00409B
:10E54000044B1B689BB203EBC000034B03445B000E
:10E5500018887047505C004004300020012910B535
:10E560002FD1254CC0002168244B89B201440B44B3
:10E570003E2A4FEA43010AD9530912F01F0F04BF84
:10E5800003F1FF339BB29B0243F4004305E05308C1
:10E5900012F0010F18BF01339B020B6023683E2A63
:10E5A0009BB21844164B03444FEA43031CD951094C
:10E5B000D00604BF01F1FF3189B2890241F4004164
:10E5C00017E0022917D10C49C0000C680B4BA4B20C
:10E5D000044423445B001A600B689BB21844084B48
:10E5E00003445B001A6010BD5108D20748BF0131D7
:10E5F0008902196010BD10BD505C0040023000203F
:10E600000630002001291BD1134B3E2A1B689BB208
:10E6100003EBC000114B03444FEA430109D95309EE
:10E62000D00604BF03F1FF339BB29B0243F40043C7
:10E6300004E05308D20748BF01339B020B607047C8
:10E64000022908D1044B1B689BB203EBC000034BAB
:10E6500003445B001A607047505C004002300020A9
:10E6600001291BD1134B3E2A1B689BB203EBC00050
:10E67000114B03444FEA430109D95309D00604BFA3
:10E6800003F1FF339BB29B0243F4004304E05308C1
:10E69000D20748BF01339B020B607047022908D1A3
:10E6A000044B1B689BB203EBC000034B03445B00AD
:10E6B0001A607047505C004006300020054B1B6814
:10E6C0009BB203EBC000044B03445B001868C0F32B
:10E6D00009007047505C004002300020054B1B6869
:10E6E0009BB203EBC000044B03445B001868C0F30B
:10E6F00009007047505C0040063000200D4AC00001
:10E7000013689BB2C1180C4B0B445B001B8813F4BD
:10E710007C4F0DD113689BB21844084B03445B0037
:10E720001B88C3F30903002B0CBF00200220704795
:10E7300001207047505C004006300020023000206D
:10E7400001290BD1800000F1804000F5B84002683B
:10E7500048F68F73134043F040030CE002290BD1BD
:10E76000800000F1804000F5B840026848F68F73E1
:10E77000134043F480430360704741EA0020704730
:10E78000C3B2000A40EA0320704700BF81F0004195
:10E7900002E000BF83F0004330B54FEA41044FEA86
:10E7A000430594EA050F08BF90EA020F1FBF54EA21
:10E7B000000C55EA020C7FEA645C7FEA655C00F0BD
:10E7C000E2804FEA5454D4EB5555B8BF6D420CDD8E
:10E7D0002C4480EA020281EA030382EA000083EA11
:10E7E000010180EA020281EA0303362D88BF30BDB1
:10E7F00011F0004F4FEA01314FF4801C4CEA113107
:10E8000002D0404261EB410113F0004F4FEA033365
:10E810004CEA133302D0524263EB430394EA050FF0
:10E8200000F0A780A4F10104D5F1200E0DDB02FA5F
:10E830000EFC22FA05F2801841F1000103FA0EF2F3
:10E84000801843FA05F359410EE0A5F120050EF1B9
:10E85000200E012A03FA0EFC28BF4CF0020C43FAEA
:10E8600005F3C01851EBE37101F0004507D54FF0F7
:10E87000000EDCF1000C7EEB00006EEB0101B1F547
:10E88000801F1BD3B1F5001F0CD349085FEA30008D
:10E890004FEA3C0C04F101044FEA445212F5800F98
:10E8A00080F09A80BCF1004F08BF5FEA500C50F135
:10E8B000000041EB045141EA050130BD5FEA4C0C18
:10E8C000404141EB010111F4801FA4F10104E9D1A1
:10E8D00091F0000F04BF01460020B1FA81F308BF98
:10E8E0002033A3F10B03B3F120020CDA0C3208DD64
:10E8F00002F1140CC2F10C0201FA0CF021FA02F13F
:10E900000CE002F11402D8BFC2F1200C01FA02F1AE
:10E9100020FA0CFCDCBF41EA0C019040E41AA2BFD3
:10E9200001EB0451294330BD6FEA04041F3C1CDA9B
:10E930000C340EDC04F11404C4F1200220FA04F0BB
:10E9400001FA02F340EA030021FA04F345EA030165
:10E9500030BDC4F10C04C4F1200220FA02F001FA27
:10E9600004F340EA0300294630BD21FA04F02946A9
:10E9700030BD94F0000F83F4801306BF81F4801142
:10E980000134013D4EE77FEA645C18BF7FEA655CB5
:10E9900029D094EA050F08BF90EA020F05D054EA87
:10E9A000000C04BF1946104630BD91EA030F1EBF8C
:10E9B0000021002030BD5FEA545C05D14000494190
:10E9C00028BF41F0004130BD14F580043CBF01F583
:10E9D000801130BD01F0004545F0FE4141F4700169
:10E9E0004FF0000030BD7FEA645C1ABF1946104644
:10E9F0007FEA655C1CBF0B46024650EA013406BF45
:10EA000052EA033591EA030F41F4002130BD00BF03
:10EA100090F0000F04BF0021704730B54FF48064C0
:10EA200004F132044FF000054FF0000150E700BF41
:10EA300090F0000F04BF0021704730B54FF48064A0
:10EA400004F1320410F0004548BF40424FF000018D
:10EA50003EE700BF42004FEAE2014FEA31014FEAD0
:10EA600002701FBF12F07F4393F07F4F81F060511F
:10EA7000704792F0000F14BF93F07F4F704730B58E
:10EA80004FF4607401F0004521F0004120E700BF21
:10EA900050EA010208BF704730B54FF000050AE0A8
:10EAA00050EA010208BF704730B511F0004502D5A9
:10EAB000404261EB41014FF4806404F132045FEAAB
:10EAC000915C3FF4DCAE4FF003025FEADC0C18BF50
:10EAD00003325FEADC0C18BF033202EBDC02C2F146
:10EAE000200300FA03FC20FA02F001FA03FE40EAD8
:10EAF0000E0021FA02F11444C1E600BF70B54FF0D8
:10EB0000FF0C4CF4E06C1CEA11541DBF1CEA1355B9
:10EB100094EA0C0F95EA0C0F00F0DEF82C4481EA21
:10EB2000030621EA4C5123EA4C5350EA013518BF41
:10EB300052EA033541F4801143F4801338D0A0FB2E
:10EB400002CE4FF00005E1FB02E506F00042E0FBDB
:10EB500003E54FF00006E1FB03569CF0000F18BFE1
:10EB60004EF0010EA4F1FF04B6F5007F64F5407489
:10EB700004D25FEA4E0E6D4146EB060642EAC6211C
:10EB800041EA55514FEAC52040EA5E504FEACE2E89
:10EB9000B4F1FD0C88BFBCF5E06F1ED8BEF1004F8C
:10EBA00008BF5FEA500E50F1000041EB045170BD08
:10EBB00006F0004646EA010140EA020081EA03014C
:10EBC000B4EB5C04C2BFD4EB0C0541EA045170BD48
:10EBD00041F480114FF0000E013C00F3AB8014F1C2
:10EBE000360FDEBF002001F0004170BDC4F100040B
:10EBF000203C35DA0C341BDC04F11404C4F120058C
:10EC000000FA05F320FA04F001FA05F240EA0200E6
:10EC100001F0004221F0004110EBD37021FA04F61C
:10EC200042EB06015EEA430E08BF20EAD37070BDD6
:10EC3000C4F10C04C4F1200500FA04F320FA05F035
:10EC400001FA04F240EA020001F0004110EBD37037
:10EC500041F100015EEA430E08BF20EAD37070BDA7
:10EC6000C4F1200500FA05F24EEA020E20FA04F380
:10EC700001FA05F243EA020321FA04F001F000412F
:10EC800021FA04F220EA020000EBD3705EEA430EA0
:10EC900008BF20EAD37070BD94F0000F0FD101F0CF
:10ECA0000046400041EB010111F4801F08BF013C08
:10ECB000F7D041EA060195F0000F18BF704703F046
:10ECC0000046520043EB030313F4801F08BF013DCD
:10ECD000F7D043EA0603704794EA0C0F0CEA135589
:10ECE00018BF95EA0C0F0CD050EA410618BF52EA43
:10ECF0004306D1D181EA030101F000414FF0000049
:10ED000070BD50EA410606BF1046194652EA430656
:10ED100019D094EA0C0F02D150EA013613D195EACA
:10ED20000C0F05D152EA03361CBF104619460AD112
:10ED300081EA030101F0004141F0FE4141F470011C
:10ED40004FF0000070BD41F0FE4141F4780170BD0C
:10ED500070B54FF0FF0C4CF4E06C1CEA11541DBF71
:10ED60001CEA135594EA0C0F95EA0C0F00F0A7F873
:10ED7000A4EB050481EA030E52EA03354FEA0131A0
:10ED800000F088804FEA03334FF0805545EA1313B3
:10ED900043EA12634FEA022245EA111545EA10657B
:10EDA0004FEA00260EF000419D4208BF964244F112
:10EDB000FD0404F5407402D25B084FEA3202B61A31
:10EDC00065EB03055B084FEA32024FF480104FF405
:10EDD000002CB6EB020E75EB030E22BFB61A754679
:10EDE00040EA0C005B084FEA3202B6EB020E75EB0C
:10EDF000030E22BFB61A754640EA5C005B084FEA74
:10EE00003202B6EB020E75EB030E22BFB61A754640
:10EE100040EA9C005B084FEA3202B6EB020E75EB4B
:10EE2000030E22BFB61A754640EADC0055EA060E0C
:10EE300018D04FEA051545EA16754FEA06164FEA4F
:10EE4000C30343EA52734FEAC2025FEA1C1CC0D1FB
:10EE500011F4801F0BD141EA00014FF000004FF088
:10EE6000004CB6E711F4801F04BF01430020B4F149
:10EE7000FD0C88BFBCF5E06F3FF6AFAEB5EB030C01
:10EE800004BFB6EB020C5FEA500C50F1000041EBFE
:10EE9000045170BD0EF0004E4EEA113114EB5C04CB
:10EEA000C2BFD4EB0C0541EA045170BD41F480119E
:10EEB0004FF0000E013C90E645EA060E8DE60CEAA6
:10EEC000135594EA0C0F08BF95EA0C0F3FF43BAFC3
:10EED00094EA0C0F0AD150EA01347FF434AF95EA7A
:10EEE0000C0F7FF425AF104619462CE795EA0C0F5E
:10EEF00006D152EA03353FF4FDAE1046194622E72B
:10EF000050EA410618BF52EA43067FF4C5AE50EA04
:10EF100041047FF40DAF52EA43057FF4EBAE12E7F4
:10EF20004FF0FF3C06E000BF4FF0010C02E000BFD5
:10EF30004FF0010C4DF804CD4FEA410C7FEA6C5CB8
:10EF40004FEA430C18BF7FEA6C5C1BD001B050EA5B
:10EF5000410C0CBF52EA430C91EA030F02BF90EA46
:10EF6000020F0020704710F1000F91EA030F58BF05
:10EF7000994208BF90422CBFD8176FEAE37040F067
:10EF8000010070474FEA410C7FEA6C5C02D150EA05
:10EF9000013C07D14FEA430C7FEA6C5CD6D152EAC0
:10EFA000033CD3D05DF8040B704700BF8446104685
:10EFB00062468C461946634600E000BF01B5FFF784
:10EFC000B7FF002848BF10F1000F01BD4DF808ED54
:10EFD000FFF7F4FF0CBF012000205DF808FB00BF25
:10EFE0004DF808EDFFF7EAFF34BF012000205DF87F
:10EFF00008FB00BF4DF808EDFFF7E0FF94BF0120CC
:10F0000000205DF808FB00BF4DF808EDFFF7CEFFCC
:10F0100094BF012000205DF808FB00BF4DF808ED0B
:10F02000FFF7C4FF34BF012000205DF808FB00BFDC
:10F030004FEA410212F5001215D211D56FF4787320
:10F04000B3EB625212D94FEAC12343F0004343EAC3
:10F05000505311F0004F23FA02F018BF404270479E
:10F060004FF00000704750EA013005D111F0004028
:10F0700008BF6FF0004070474FF00000704700BFBE
:10F080004FEA4102B2F1E04324BFB3F5001CDCF1CA
:10F09000FE5C0DD901F0004C4FEAC0024CEA507002
:10F0A000B2F1004F40EB830008BF20F00100704731
:10F0B00011F0804F21D113F13872BCBF01F0004034
:10F0C000704741F480114FEA5252C2F11802C2F166
:10F0D000200C10FA0CF320FA02F018BF40F00100E7
:10F0E0004FEAC1234FEAD32303FA0CFC40EA0C0099
:10F0F00023FA02F34FEA4303CCE77FEA625307D1D6
:10F1000050EA01331EBF4FF0FE4040F4400070470C
:10F1100001F0004040F0FE4040F40000704700BFA6
:10F1200080F0004002E000BF81F0004142001FBFBC
:10F130005FEA410392EA030F7FEA226C7FEA236CC5
:10F140006AD04FEA1262D2EB1363C1BFD2184140BA
:10F1500048404140B8BF5B42192B88BF704710F050
:10F16000004F40F4000020F07F4018BF404211F0F3
:10F17000004F41F4000121F07F4118BF494292EA5B
:10F18000030F3FD0A2F1010241FA03FC10EB0C0087
:10F19000C3F1200301FA03F100F0004302D5494214
:10F1A00060EB4000B0F5000F13D3B0F1807F06D3C1
:10F1B00040084FEA310102F10102FE2A51D2B1F1B9
:10F1C000004F40EBC25008BF20F0010040EA0300AE
:10F1D0007047490040EB000010F4000FA2F101025B
:10F1E000EDD1B0FA80FCACF1080CB2EB0C0200FAE5
:10F1F0000CF0AABF00EBC25052421843BCBFD04033
:10F200001843704792F0000F81F4000106BF80F4AC
:10F2100000000132013BB5E74FEA41037FEA226C6F
:10F2200018BF7FEA236C21D092EA030F04D092F03A
:10F23000000F08BF0846704790EA010F1CBF00206E
:10F24000704712F07F4F04D1400028BF40F00040CB
:10F25000704712F100723CBF00F50000704700F0EB
:10F26000004343F0FE4040F4000070477FEA226212
:10F2700016BF08467FEA23630146420206BF5FEAE3
:10F28000412390EA010F40F4800070474FF00003E3
:10F2900004E000BF10F0004348BF40425FEA000CAA
:10F2A00008BF704743F0964301464FF000001CE052
:10F2B00050EA010208BF70474FF000030AE000BFA8
:10F2C00050EA010208BF704711F0004302D54042E6
:10F2D00061EB41015FEA010C02BF84460146002058
:10F2E00043F0B64308BFA3F18053A3F50003BCFA73
:10F2F0008CF2083AA3EBC25310DB01FA02FC634420
:10F3000000FA02FCC2F12002BCF1004F20FA02F226
:10F3100043EB020008BF20F00100704702F1200219
:10F3200001FA02FCC2F1200250EA4C0021FA02F27A
:10F3300043EB020008BF20EADC7070474FF0FF0C7F
:10F340001CEAD0521EBF1CEAD15392EA0C0F93EA7A
:10F350000C0F6FD01A4480EA010C400218BF5FEA1C
:10F3600041211ED04FF0006343EA501043EA51118F
:10F37000A0FB01310CF00040B1F5000F3EBF490089
:10F3800041EAD3715B0040EA010062F17F02FD2A8D
:10F390001DD8B3F1004F40EBC25008BF20F0010070
:10F3A000704790F0000F0CF0004C08BF49024CEA87
:10F3B000502040EA51207F3AC2BFD2F1FF0340EA19
:10F3C000C250704740F400004FF00003013A5DDC8A
:10F3D00012F1190FDCBF00F000407047C2F10002CB
:10F3E000410021FA02F1C2F1200200FA02FC5FEAB8
:10F3F000310040F1000053EA4C0308BF20EADC7002
:10F40000704792F0000F00F0004C02BF400010F473
:10F41000000F013AF9D040EA0C0093F0000F01F020
:10F42000004C02BF490011F4000F013BF9D041EA42
:10F430000C018FE70CEAD15392EA0C0F18BF93EA44
:10F440000C0F0AD030F0004C18BF31F0004CD8D16E
:10F4500080EA010000F00040704790F0000F17BFF5
:10F4600090F0004F084691F0000F91F0004F14D03B
:10F4700092EA0C0F01D142020FD193EA0C0F03D193
:10F480004B0218BF084608D180EA010000F0004096
:10F4900040F0FE4040F40000704740F0FE4040F471
:10F4A000400070474FF0FF0C1CEAD0521EBF1CEA10
:10F4B000D15392EA0C0F93EA0C0F69D0A2EB03022E
:10F4C00080EA010C49024FEA402037D04FF08053C8
:10F4D00043EA111143EA10130CF000408B4238BF8D
:10F4E0005B0042F17D024FF4000C8B4224BF5B1A9B
:10F4F00040EA0C00B3EB510F24BFA3EB510340EAE9
:10F500005C00B3EB910F24BFA3EB910340EA9C0096
:10F51000B3EBD10F24BFA3EBD10340EADC001B0106
:10F5200018BF5FEA1C1CE0D1FD2A3FF650AF8B42AA
:10F5300040EBC25008BF20F0010070470CF0004CB7
:10F540004CEA50207F32C2BFD2F1FF0340EAC250E2
:10F55000704740F400004FF00003013A37E792F0A3
:10F56000000F00F0004C02BF400010F4000F013A01
:10F57000F9D040EA0C0093F0000F01F0004C02BFFC
:10F58000490011F4000F013BF9D041EA0C0195E765
:10F590000CEAD15392EA0C0F08D142027FF47DAFFE
:10F5A00093EA0C0F7FF470AF084676E793EA0C0FEE
:10F5B00004D14B023FF44CAF08466EE730F0004CEC
:10F5C00018BF31F0004CCAD130F000427FF45CAF7C
:10F5D00031F000437FF43CAF5FE700BF4FF0FF3CEA
:10F5E00006E000BF4FF0010C02E000BF4FF0010C3D
:10F5F0004DF804CD4FEA40024FEA41037FEA226C06
:10F6000018BF7FEA236C11D001B052EA530C18BF27
:10F6100090EA010F58BFB2EB030088BFC81738BF8C
:10F620006FEAE17018BF40F0010070477FEA226C7A
:10F6300002D15FEA402C05D17FEA236CE4D15FEA76
:10F64000412CE1D05DF8040B704700BF84460846AA
:10F650006146FFE70FB5FFF7C9FF002848BF10F16B
:10F66000000F0FBD4DF808EDFFF7F4FF0CBF0120B0
:10F6700000205DF808FB00BF4DF808EDFFF7EAFF3A
:10F6800034BF012000205DF808FB00BF4DF808EDF5
:10F69000FFF7E0FF94BF012000205DF808FB00BFEA
:10F6A0004DF808EDFFF7D2FF94BF012000205DF870
:10F6B00008FB00BF4DF808EDFFF7C8FF34BF01207D
:10F6C00000205DF808FB00BF42000ED2B2F1FE4FF1
:10F6D0000BD34FF09E03B3EB126209D44FEA002321
:10F6E00043F0004323FA02F070474FF000007047E8
:10F6F00012F1610F01D1420202D14FF0FF30704789
:10F700004FF00000704700BF73B96AB9002908BF05
:10F710000028BCBF00204FF00041C4BF6FF0004183
:10F720004FF0FF3000F03CB882B0EC462DE90050BD
:10F7300000F006F8DDF804E002B00CBC704700BF32
:10F740002DE9704F089E14461D468046894600F0FC
:10F7500029F804FB01F3A4FB00AB00FB0532934442
:10F76000B8EB0A0869EB0B09C6E90089BDE8708FA0
:10F770002DE9704F089E14461D468046894600F0CC
:10F7800061F900FB05F5A0FB04AB04FB0154A344A5
:10F79000B8EB0A0869EB0B09C6E90089BDE8708F70
:10F7A000704700BF00292DE9F00FC0F2A1800024AE
:10F7B000002BC0F29880154606460F46002B3FD11D
:10F7C0008A4258D9B2FA82F34BB1C3F1200201FA4E
:10F7D00003F720FA02F29D4000FA03F61743290CC2
:10F7E000B7FBF1F201FB1277A8B200FB02F34FEA7C
:10F7F000164C4CEA0747BB4209D97F1902F1FF3C7E
:10F8000080F00581BB4240F20281023A2F44FF1A88
:10F81000B7FBF1F301FB137100FB03F0B6B246EA4C
:10F820000141884208D9491903F1FF3780F0F1807E
:10F83000884240F2EE80023B43EA0242002303E0AA
:10F840008B420AD900231A461046194614B1404289
:10F8500061EB4101BDE8F00F7047B3FA83F8B8F1EE
:10F86000000F40F088808B4202D3824200F2E28097
:10F8700000230122E8E712B90123B3FBF2F5B5FA40
:10F8800085F2002A3AD17F1B280C1FFA85FC012340
:10F89000B7FBF0F100FB11770CFB01F24FEA1648C1
:10F8A00048EA0747BA4207D97F1901F1FF3802D267
:10F8B000BA4200F2C4804146BF1AB7FBF0F200FB27
:10F8C00012700CFB02FCB6B246EA0040844507D930
:10F8D000401902F1FF3702D2844500F2AE803A4669
:10F8E00042EA0142B0E7E443524263EB430362E77A
:10F8F000404261EB41014FF0FF3459E79540C2F1BE
:10F90000200927FA09F126FA09F99740280CB1FBDA
:10F91000F0F800FB18111FFA85FC0CFB08F349EA0C
:10F9200007094FEA194747EA01418B4206FA02F6F6
:10F9300008D9491908F1FF327AD28B4278D9A8F157
:10F9400002082944C91AB1FBF0F300FB13170CFBA2
:10F9500003F21FFA89F949EA0747BA4207D97F1922
:10F9600003F1FF3160D2BA425ED9023B2F44BF1A85
:10F9700043EA08438CE7C8F1200225FA02F103FAB2
:10F9800008FC27FA02F320FA02F207FA08F741EA24
:10F990000C0C4FEA1C49B3FBF9F109FB11331FFAB8
:10F9A0008CFA0AFB01FB17433A0C42EA03439B45DE
:10F9B00005FA08F008D913EB0C0301F1FF3235D238
:10F9C0009B4533D902396344CBEB0303B3FBF9F214
:10F9D00009FB12330AFB02FABFB247EA0347BA45F2
:10F9E00008D917EB0C0702F1FF331BD2BA4519D91E
:10F9F000023A674442EA0145A5FB0001CAEB07074A
:10FA00008F424FF000030AD305D02A461CE7624616
:10FA1000FDE63B4610E706FA08F68642F5D26A1E76
:10FA2000002311E71A46E5E70B46A0E71146CBE7AE
:10FA3000904687E74346424606E7023A50E70239D6
:10FA40002F4439E72DE9F00F144605460E46002BEA
:10FA500043D18A4253D9B2FA82F757B1C7F120068F
:10FA600020FA06F601FA07F302FA07F400FA07F59E
:10FA70001E43210CB6FBF1F201FB1266A0B200FBA3
:10FA800002F32F0C47EA0646B34209D9361902F1B0
:10FA9000FF3780F0FD80B34240F2FA80023A2644FC
:10FAA000F61AB6FBF1F301FB136100FB03F0ADB2F4
:10FAB00045EA0141884208D9091903F1FF3680F06F
:10FAC000E980884240F2E680023B43EA024200239A
:10FAD00010461946BDE8F00F70478B424CD8B3FA78
:10FAE00083F6002E4FD18B4202D3824200F2DD809A
:10FAF000BDE8F00F0023012210461946704712B9E5
:10FB00000124B4FBF2F4B4FA84F2002A40F08280BB
:10FB1000091B260CA7B20123B1FBF6F006FB10115E
:10FB200007FB00F24FEA154C4CEA01418A4207D923
:10FB3000091900F1FF3C02D28A4200F2C8806046F7
:10FB4000891AB1FBF6F206FB121107FB02F7ADB200
:10FB500045EA0145AF4208D92C1902F1FF3180F086
:10FB60009B80A74240F29880023A42EA0042104647
:10FB70001946BDE8F00F704700231A461046194693
:10FB8000BDE8F00F7047C6F1200522FA05F703FA29
:10FB900006F421FA05F301FA06FB20FA05F53C43C9
:10FBA0004FEA1448B3FBF8FC08FB1C331FFA84F936
:10FBB00009FB0CFA45EA0B0B4FEA1B4545EA0343E8
:10FBC0009A4502FA06F204D91B190CF1FF356FD3DE
:10FBD000AC46CAEB0303B3FBF8F508FB153309FB8E
:10FBE00005F91FFA8BFB4BEA0347B94504D93F19C6
:10FBF00005F1FF3362D31D4645EA0C4CACFB0223F2
:10FC0000C9EB07079F424FF000054AD346D0624632
:10FC10002B465DE79440C2F1200921FA09FC91408E
:10FC200020FA09F9260CBCFBF6F806FB18CCA7B2A3
:10FC300007FB08F349EA01094FEA194141EA0C4C74
:10FC4000634500FA02F509D91CEB040C08F1FF32F8
:10FC50003BD2634539D9A8F10208A444C3EB0C0C8C
:10FC6000BCFBF6F306FB13C107FB03F21FFA89F98D
:10FC700049EA01418A4207D9091903F1FF3022D22A
:10FC80008A4220D9023B2144891A43EA084343E7C8
:10FC90003A4605E7334618E70A4666E7B040904221
:10FCA000B5D20CF1FF32002312E7334632460FE79C
:10FCB0009A458DD9ACF1020C23448AE7B9459AD90B
:10FCC000023D274498E70346DEE79046C6E7023840
:10FCD000214435E773B5524EFCF716FA00244FF471
:10FCE00080303470FCF72EFAFCF77CFB01280546C7
:10FCF00025D11020FBF728FD2046FCF771FA20469D
:10FD0000FCF782FA2046FCF775FA4FF480304FF486
:10FD10008021FCF743FA2846FCF74AFA3920FCF721
:10FD20004DFB0028FAD00120FBF7F6FC0120FCF780
:10FD300045FAFCF74DFA0428FBD101233370042067
:10FD40000121FCF7F9FA4FF48073ADF80430032376
:10FD500001A98DF80630334818238DF80730FBF7DA
:10FD600074FF0620FCF724FB01200146FCF7E4FAAF
:10FD70004FF0C0500121FCF7EBFA4FF480414FF0F7
:10FD80000060FCF70DF9284C4FF44070FCF75EF86A
:10FD9000F4F7F6F9F4F756FD01232370234A244BB8
:10FDA00024491360244A254D1160254A1360F4F755
:10FDB0003FFBF8F7DDFAF8F7BDFAF8F799F8F4F732
:10FDC00085FA2878F8F708F9E878F8F74BFA2378F5
:10FDD0000BB1F8F73FFEF9F7ADF8F4F7B7FCFAF717
:10FDE000D1FEF7F749FAF8F7ABFEF9F7DFFB154B51
:10FDF0004FF480625A61F7F741FBF9F7E3FBF8F73C
:10FE0000A0FEF4F7EDFCF4F70FFD0028F3D0F9F7AE
:10FE100091F8F7F731FAF9F7C9FBF8F7A9FEEAE725
:10FE2000240F002000080140500E0020680E002022
:10FE3000B982000883880008300F002008000020E5
:10FE4000C40E0020000C014000210A2200F0ACB8D2
:10FE50000F4B30B405461C6802E0D01A16D1ABB186
:10FE600015F8013BE21850781A4600F0030001280B
:10FE700008BF03F1200211F8013BE018407800F0C0
:10FE800003000128E9D12033D01AE9D030BC7047F3
:10FE90005C0500202DE9F00F424C82B0D4F800C080
:10FEA00001900E4600E02646344614F8015B0CEB48
:10FEB0000500407800F0080000F0FF0A0028F2D1A9
:10FEC0002D2D5BD02B2D04BF7578B41C33F01000A2
:10FED0003CD09946BAF1000F0CBF6FF0004B4FF0C9
:10FEE000004BBBFBF9F8002709FB18BB38460CE0B8
:10FEF000303DAB4219DD7E1C05D0404523D820D0D3
:10FF000009FB0050012714F8015B0CEB050676781D
:10FF100016F0040FECD116F0030606D0012E14BF24
:10FF200057263726AD1BAB42E5DC7B1C15D0BAF15A
:10FF3000000F21D10AB1EFB9116002B0BDE8F00F96
:10FF400070475D45DCDD4FF0FF37DCE7302D1AD020
:10FF5000002BBED10A239946BCE70199BAF1000FE4
:10FF60004FF022030CBF6FF000404FF000400B60D9
:10FF7000002AE2D0611EDFE74042DBE7B41C75785F
:10FF80004FF0010AA2E7207800F0DF00582803D0E4
:10FF9000002B9ED108239CE71023657899460234F4
:10FFA00098E700BF5C05002030B4044C0D461346B2
:10FFB00001462A46206830BCFFF76CBF5805002078
:10FFC0002DE9F0418AB004460D4600F06DF8DFF8E7
:10FFD000D080064698F900300F4601330BD02046FA
:10FFE000294600F059FA30B1204629460022002364
:10FFF000FFF714F820B1304639460AB0BDE8F08169
:020000040801F1
:10000000234B98F800600890CDE90245CDE90445FE
:10001000019346BB1F4B4FF06042CDE906232046BB
:10002000294600220023FEF7D1FF70B102239E4231
:10003000009322D0684600F057FAF0B1089B0BBB42
:10004000DDE906010AB0BDE8F0810123022E00932C
:100050000ED0684600F048FA50B10F4800F046FA5A
:10006000CDE90601EAE70D4B0022CDE90623D6E7EC
:1000700000F042FA21230360EFE700F03DFA22236B
:100080000360DBE700F038FA089B0360D8E700BFA5
:100090002C080108FFFFEFC7300801080000F0FF3F
:1000A00060050020000000002DE9F04FB1F5801F31
:1000B00087B002460B460F465BDA21F00046064346
:1000C00000F0F5800029C0F2A4810022B24BFEF7B7
:1000D00015FD0F460B46B14902468F426FF03505BC
:1000E0004BDCC7F3130606F5152101F6647101F424
:1000F000801484F07F5181F4401141EA06031046D8
:1001000019460022A64BFEF745FB4FEA2758B31CC1
:10011000A8F2FF38C3F31303A844022B08EB1458CA
:1001200082468B464FF000022EDC0023FEF74EFF86
:10013000002800F0C580B8F1000F00F07181404642
:10014000FEF776FC80A3D3E9002306460F46FEF7B0
:10015000D5FC7FA3D3E9002304460D46304639463B
:10016000FEF7CCFC02460B4620462946FEF714FB60
:1001700007E08A4900258F42B3DD10461946FEF795
:100180000BFB07B0BDE8F08F4FF08043FEF704FB98
:1001900002460B4650465946FEF7DAFDCDE902010C
:1001A0004046FEF745FCCDE90401DDE902010246C7
:1001B0000B46FEF7A3FC02460B46CDE90001FEF715
:1001C0009DFC65A3D3E9002304460D46FEF796FC8B
:1001D00063A3D3E90023FEF7DFFA22462B46FEF79E
:1001E0008DFC61A3D3E90023FEF7D6FA22462B4605
:1001F000FEF784FC5EA3D3E90023FEF7CDFADDE928
:100200000023FEF77BFC5CA3D3E90023CDE90001CA
:1002100020462946FEF772FC59A3D3E90023FEF7D6
:10022000BBFA22462B46FEF769FC57A3D3E900230D
:10023000FEF7B2FA22462B46FEF760FC0B4602465A
:10024000DDE90001FEF7A8FAA6F5C223C6F5D72618
:10025000A3F27A4351361E43002E04460D4657DD65
:100260000022504B50465946FEF748FC52465B462A
:10027000FEF744FC06460F46B8F1000F40F09680AA
:1002800022462B46FEF788FADDE90223FEF736FC0C
:1002900002460B4630463946FEF77CFA02460B46CC
:1002A00050465946FEF776FA07B0BDE8F08F0022B7
:1002B000002300203C49FEF74BFD07B0BDE8F08F5E
:1002C00052465B4650465946FEF718FC30A3D3E928
:1002D000002304460D4650465946FEF70FFC0246E1
:1002E0000B4600202F49FEF755FA02460B462046E2
:1002F0002946FEF703FC04460D46B8F1000F40F016
:1003000092805046594622462B46FEF743FA38E77C
:10031000B8F1000F00F0AB800BA3D3E90023DDE9B7
:100320000401FEF7EBFB22462B4606460F465046DD
:100330005946FEF72FFADDE90223FEF7DFFB0446FC
:100340000D46DDE904017CE00000E0FE422EE63FC0
:10035000763C7935EF39EA3D44523EDF12F1C23F37
:10036000DE03CB966446C73F599322942449D23F7B
:10037000935555555555E53F9FC678D0099AC33FCB
:10038000AF788E1DC571CC3F04FA97999999D93FE2
:10039000555555555555D53F00005043FFFFEF7F4C
:1003A0000000F03F0000E03F000050C336A3D3E957
:1003B0000023DDE90401FEF7A1FB224680468946C1
:1003C0002B4630463946FEF7E7F9DDE90223FEF712
:1003D00095FB2FA3D3E9002304460D46DDE9040174
:1003E000FEF78CFB02460B4620462946FEF7D4F961
:1003F00002460B4630463946FEF7CCF952465B467C
:10040000FEF7C8F902460B4640464946FEF7C2F9D8
:10041000B7E6FEF7BFF900220023FEF799FCB0E62D
:1004200000200021ADE64046FEF702FB16A3D3E90B
:10043000002380468946FEF761FB06460F4640468C
:10044000494613A3D3E90023FEF758FB02460B46A7
:1004500020462946FEF79EF952465B46FEF79AF97A
:1004600002460B4630463946FEF794F989E60246C5
:100470000B4650465946FEF78DF9DDE90223FEF79B
:100480003DFB0BE7AFF300800000E0FE422EE63FAD
:10049000763C7935EF39EA3D31F0004310B408D0AD
:1004A0000F4AA3F5801494420AD804205DF8044B47
:1004B000704700280CBF022003205DF8044B7047F2
:1004C000B3F5801F01D20320F7E7064A934201D01B
:1004D0000020F2E7D0F1010038BF0020EDE700BFB7
:1004E000FFFFDF7F0000F07F002070470020014900
:1004F000704700BF0000F87F014B1868704700BFCD
:1005000058050020F4010000640000000180080884
:100510000000000000640000000000000000000077
:10052000C80000000000000000000000010003E817
:100530000000000000000003E800000000000200CE
:10054000FA0600030000000000370600000000006B
:100550000000000032035400720069006E00610068
:100560006D00690063002000530074006500700096
:10057000700065007200200044006500760069008C
:1005800063006500200026035400720069006E00BD
:1005900061006D00690063004D006F007400690028
:1005A0006F006E002000430074006C000403090417
:1005B00009024300020100C03209040000010202E6
:1005C0000100052400100105240100010424020299
:1005D0000524060001070582030800FF0904010045
:1005E000020A00000007050302400000070581021F
:1005F00040000012011001020000403C2A000101ED
:100600002401020301524F5200000106524F4C00D8
:100610000002064D5354000003024D5650000004E2
:10062000075341500000050747415000000603539F
:1006300054415000070352534150000803534750A0
:100640000000090747475000000A03535447500071
:100650000B0352534750000C0352465300000D0346
:1006600053494F00000E0747494F00000F03534105
:100670004300001D0753434F00001E0747434F0030
:10068000001F0343434F0000200341434F00002756
:1006900003554630000040075546310000410755DC
:1006A00046320000420755463300004307554634A2
:1006B0000000440755463500004507554636000002
:1006C00046075546370000470752554E0000810542
:1006D00053544F5000800042494E00008B000000F0
:1006E00000000000000000000001020304010203FA
:1006F000040607080902040608313138315631333F
:1007000036004142530052454C00434F4F52440083
:1007100053544152540053544F5000535441545574
:100720005300000043000000002020202020202053
:100730002020282828282820202020202020202091
:1007400020202020202020202088101010101010A1
:1007500010101010101010101004040404040404ED
:100760000404041010101010101041414141414187
:100770000101010101010101010101010101010169
:100780000101010110101010101042424242424279
:100790000202020202020202020202020202020239
:1007A00002020202101010102000000000000000E1
:1007B0000000000000000000000000000000000039
:1007C0000000000000000000000000000000000029
:1007D0000000000000000000000000000000000019
:1007E0000000000000000000000000000000000009
:1007F00000000000000000000000000000000000F9
:1008000000000000000000000000000000000000E8
:1008100000000000000000000000000000000000D8
:100820000000000000000000000000006C6F670086
:0408300000000000C4
:0808340070EFFF7F01000000DE
:10083C00F906010800010000000102000008000098
:10084C000100000002000000000000000000000099
:10085C00000000000000000000000000000000008C
:10086C00000000000000000000000000000000007C
:10087C00000000000000000000C2010000000800A1
:10088C002D890008F1860008F1850008058600080E
:10089C00078600086186000885860008CD87000859
:1008AC00D9870008E5870008000000004000000020
:1008BC00F305010812000000B00501084300000018
:1008CC00AC050108040000008605010826000000A4
:1008DC005405010832000000140100201A00000029
:1008EC0001000000C1DD0008CD850008C1DD000855
:1008FC00C1DD0008C1DD0008C1DD0008C1DD000854
:10090C00C1DD0008E585000804010000C1DD000818
:10091C00C1DD0008C5860008C1DD0008C1DD000886
:10092C00C1DD0008C1DD0008C1850008C1DD00087B
:10093C00C1DD0008C1DD0008C1DD0008C1DD000813
:10094C00C1DD00081A0354004D004300530054004D
:10095C0045005000000000000000000000000000F6
:10096C00000000001C04002084040020EC04002083
:10097C00000000000000000000000000000000006B
:10098C00000000000000000000000000000000005B
:10099C000000000024070108000000000000000017
:1009AC00000000000000000000000000000000003B
:1009BC00000000000000000000000000000000002B
:1009CC00000000000000000000000000000000001B
:1009DC00000000000000000000000000000000000B
:1009EC0000000000000000000000000000000000FB
:1009FC0000000000000000000000000000000000EB
:100A0C0000000000000000000100000000000000D9
:100A1C000E33CDAB34126DE6ECDE05000B0000009E
:100A2C0000000000000000000000000000000000BA
:100A3C0000000000000000000000000000000000AA
:100A4C00000000000000000000000000000000009A
:100A5C00000000000000000000000000000000008A
:100D8C0000000000000000003001002028070108CE
:040D9C000100000052
:04000005080041109E
:00000001FF
